:020000040000FA
:1000000008740020E100000071690000D5000000C4
:1000100000000000000000000000000000000000E0
:10002000000000000000000000000000ED000000E3
:100030000000000000000000EF000000F1000000E0
:10004000F3000000F16F0000516E0000F3000000AB
:10005000C1160000F3000000F3000000F3000000F0
:10006000F3000000F300000029750000F300000019
:10007000F3000000F300000069750000F3000000C9
:10008000F3000000F300000000000000F300000097
:10009000056400008D1E0000F3000000711A0000CE
:1000A0008D140000F3000000F30000002514000090
:1000B000F3000000F3000000F3000000F300000074
:1000C0000348854600F044FD00480047AD99000014
:1000D000087400207046694608F08AFDFFF7FEFFAD
:1000E0000448804704480047FEE7FEE7FEE7FEE7D6
:1000F000FEE7FEE73D730000C100000030B50B468F
:10010000014600202022012409E00D46D5409D42F1
:1001100005D31D469540491B254695404019154677
:10012000521E002DF1DC30BD70B50024254600289C
:1001300001DA01244042002901DA01254942FFF792
:10014000DDFFAC4200D04042002C00D0494270BDDF
:10015000F0B51FB40646002082B005464024019148
:1001600000901BE0019922460F46304600F02CFC1F
:10017000049A059B801A994110D3104619462246CD
:1001800000F012FC361A8F4101972246012000210F
:10019000009F00F009FC38184D4100902046641E75
:1001A0000028DFDC019B00982946324607B0F0BDED
:1001B00003460B439B0703D009E008C9121F08C080
:1001C000042AFAD203E00B780370401C491C521E2B
:1001D000F9D27047D2B201E00270401C491EFBD236
:1001E00070470022F6E710B513460A460446194642
:1001F000FFF7F0FF204610BD30B505462A460B46F6
:1002000010781C78521C5B1C002801D0A042F7D04B
:10021000002C03D0002802D06D1CEFE7284630BD2B
:10022000421C0178401C0029FBD1801A7047032131
:10023000001D401E037812021A43491EF9D51046CC
:100240007047034610B508330722040E0902214304
:100250005B1E1C7800022043521EF6D510BD0346DB
:1002600003220870000A491C521EFAD5184670472E
:1002700070B504460D46072310700E06000A304381
:10028000090A521C5B1EF7D52046294670BDF8B5F9
:1002900002464A40D40F42004B0052085B089A4283
:1002A00002D20246084611464A0023D0C30D4A0036
:1002B000DDB2120EAD1A202D35DA49020126490AA7
:1002C000F6058A19002C00D0524220214F1B1146FE
:1002D000B9402A411018C20D9A4221D0002C17D0E3
:1002E000012D08DCDA05801AD20F8019D207DBB2A3
:1002F00000F096FBF8BDDA05801A012340001B06CA
:10030000C01880185A428018CA0F1043490007E0ED
:100310004908C2071143DA05801A8019400880187D
:1003200000F076FBF8BD61000122511A001BF7E7CF
:100330000122D2075140AAE70122D2075040A6E786
:10034000024670B54A40D30FDB0740002DD04A006B
:100350002AD0010E140E000212020919400A520A94
:100360008418E50104465443000A120A2E0450433F
:10037000A4194219200CC543AA18120C0125AD037B
:10038000521C521912047F39240400D0521C10430D
:1003900001D44000491EC2B20C06C0092018401CFE
:1003A0004008802A02D003E0002070BD40084000D1
:1003B000002900DA0020184370BD70B502464A409B
:1003C000D50F40004A00ED0740085208002814D01D
:1003D000002A12D0C40DD30D41020120C0055202E3
:1003E000490A520AE41A091812187D34914201D3BD
:1003F000641C00E04900002C01DA002070BD0023DD
:10040000914201D3891A0343400849000028F7D1DB
:1004100000290AD0914202D10121C90705E0914289
:1004200001D2012101E00121C943E005C0184019B2
:1004300000F0EEFA70BD0000F0B5074608465840DF
:1004400087B0C00F049048000E4659004008490884
:10045000BC1A884105D2384631461E4617460B461F
:1004600002465800400810434CD0300D0390400520
:100470005900400D490D0590401A0290402872DA4B
:1004800018030121000B090508430190049800920C
:10049000002805D001995242002088410092019025
:1004A000029840210A1A0199009800F07DFA054649
:1004B0000C466B4607CB00F098FAC0197141039ABD
:1004C0000E0D0023D71756401A467A40164344D0E3
:1004D000049A002A2DD0029A012A039A15DC1205EB
:1004E000C01A914101263605001C7141D20F059EAC
:1004F000D2070093019202962A46234600F0D6FACC
:1005000007B0F0BD38463146FAE71605224A0F46D5
:10051000B218C01AB74101210905001C4F4100184B
:100520007F41114618187941E20F10436D1964415B
:1005300013E0E2076D0815436408C2071443039AE9
:1005400001261205C01A91413605001C7141CE07E3
:10055000400830434908C01851412A46234600F05C
:1005600098FACDE7FFE7049801224000C117121A5C
:1005700000238B4104983146C417381AA141EEE795
:1005800030B40124E407634030BC55E730B40124A3
:10059000E407614030BC4FE70000E0FFF0B51FB456
:1005A00088B00B990998002448400999C00F490068
:1005B00049080991C0070B990090490049080B911F
:1005C00009990898A64608431CD00B990A98084335
:1005D00018D0099801244000420D4800410D0998A7
:1005E00024050003000B204309900B980003000B27
:1005F00020430B9050181C494018002201901446CB
:10060000104605E0002001460DB0F0BD032801DAD8
:10061000034600E003239C46C11A0AAE0AE05F00CD
:1006200008ADED5B4F00F75B7D430027AA187C41C6
:10063000491C5B1E6145F2DD410004AB5A522104A6
:10064000120C0A43240C401C0828DFDB019802909E
:100650000099704601910090059B049A07990698AD
:1006600000F024FAD0E700000DFCFFFFF0B50C46C7
:100670005C4085B0E40FE40703944C000026640856
:1006800059009446490802460296224321D0624608
:100690000A431ED06200570D4A000E032303550D76
:1006A000012402462C492405781B1B0B360B4018ED
:1006B00023432643614600901C46501AB44103D39D
:1006C0000098401C009002E0921800985B410028BE
:1006D00003DA0020014605B0F0BD00200121090524
:1006E0000746864611E064461D46141BB54106D3F5
:1006F0006546521BB341744607430C43A646CD07DB
:1007000040084908284392185B4105460D43EAD149
:100710001046184313D060461946504071400843B4
:1007200006D06046101AB34106D20122002306E02B
:1007300000220123DB0702E00122D243531000987C
:1007400074460105381C6141029C039D00196941F2
:1007500000F09FF9BFE70000FD030000C217C10FC2
:10076000504010B54018CA079623002100F058F9F0
:1007700010BD10B500229623114600F051F910BDAE
:100780000EB5C217C10F5040CA0740180021054BD3
:100790000293019200910A460B4600F087F903B0DC
:1007A00000BD0000330400000EB505490291002190
:1007B00000910A460B46019100F078F903B000BDA4
:1007C00033040000C20F410040020123400ADB0550
:1007D000D207090EC0187F2901DA00207047962938
:1007E00003DC9623591AC84001E096398840002A54
:1007F000F4D040427047410040020122400AD20535
:10080000090E80187F2901DA00207047962903DC41
:100810009622511AC84070479639884070470000A8
:1008200070B5CD0F4A0009030123090B1B051943BD
:100830000B4BED070024520D9A4201DA002070BDE7
:10084000074B34339A4203DC9A1A00F0BDF802E0F9
:100850000449511888402C43F1D0404270BD00003B
:10086000FF030000CDFBFFFF4A0009030123090B32
:100870001B051943094B10B5520D9A4201DA0020AD
:1008800010BD064B34339A4203DC9A1A00F09CF8F0
:1008900010BD03495118884010BD0000FF0300003F
:1008A000CDFBFFFF4A0009030123090B1B05194378
:1008B0000A4B10B5520D9A4202DA0020014610BDD3
:1008C000064B34339A4203DC9A1A00F07DF810BDCF
:1008D000034BD21800F068F810BD0000FF030000C1
:1008E000CDFBFFFFC20FD207400040080BD0C10D67
:1008F0000723DB01C91840020905400A1143C20859
:1009000040071143704700200146704710B5002989
:1009100004DB0124E40740428C412146002B04DB28
:100920001C460123DB075242A3418B4200D1824285
:1009300010BD000010B5002904DB0124E40740428B
:100940008C412146002B04DB1C460123DB0752426D
:10095000A341994200D1904210BD0000CB0FDB07AC
:10096000490010B5490802460A4307D00A0D07247A
:100970000903E401090B121B002A01DC002010BD51
:10098000C900440F0C43C100E018D205801800F0E4
:100990003FF810BD0122D207002800DB101A002901
:1009A00000DB511A8842704710B5202A04DB01464B
:1009B000203A9140002010BD914020239C1A03460C
:1009C000E3401943904010BD10B5202A04DB0846CF
:1009D000203AD040002110BD0B46D340D040202407
:1009E000A21A91400843194610BD10B5202A06DB13
:1009F000CB170846203A1041C1170B4306E00B46BF
:100A00001341D0402024A21A91400843194610BD3A
:100A1000002904DA401C490001D140084000704719
:100A200070B40024050C05D11024000402D1002963
:100A300021D01124050E01D100020834050F01D187
:100A40000001241D850F01D18000A41C002801DBBA
:100A50004000641C002908D020252E1B0D46F540BF
:100A6000A14000D001212943084301061B1B000AB5
:100A7000DB1D02D5002070BC7047DB0518188018FC
:100A80000029F8DA401C4900F5D170BC400840004C
:100A9000704710B5002B08DA0024401C6141921801
:100AA0005B411A4301D14008400010BDF0B51FB4AE
:100AB00082B005460C0003D0084607F0AFF902E00B
:100AC00007F0ACF920300246009021462846FFF797
:100AD0006BFF049B059A04460F46184311430843D5
:100AE00014D0184610431BD0009840210A1A18460B
:100AF0000599FFF769FF05460E46009A0599049887
:100B0000FFF752FF084305D0012004E02046394694
:100B100007B0F0BD0020C11705430E432C433743F7
:100B200000990E986305401A7905E40A00220C43E7
:100B3000FD0A0A3002D500200146E9E70105101937
:100B400069410C9C0D9D00196941FFF7A2FFDFE789
:100B5000064C0125064E05E0E36807CC2B430C3C10
:100B600098471034B442F7D3FFF7AEFAC0AA00009A
:100B7000E0AA000070B58C180578401C6B075B0F6D
:100B800001D10378401C2A1106D10278401C03E0F1
:100B900006780E70401C491C5B1EF9D12B0705D44A
:100BA0000023521E0DD40B70491CFAE70378401C39
:100BB000CB1A921C03E01D780D70491C5B1C521E61
:100BC000F9D5A142D8D3002070BD00000146064AE5
:100BD000106907231B0402469A4310461A460A402E
:100BE0001043014A1061704700FA0140012806D104
:100BF0000649096920221143044A116105E00349AD
:100C0000096920229143014A1161704700FA0140AD
:100C10000146054A1069000900010A07120F104336
:100C2000014A10617047000000FA0140012806D116
:100C30000649096840221143044A116005E003494E
:100C4000096840229143014A1160704700FA01404F
:100C5000012806D10649096801221143044A11609E
:100C600005E00349096849084900014A11607047D5
:100C700000FA01400146064A1068082302469A43DA
:100C8000104608220A401043014A106070470000D5
:100C900000FA01400146064A1068042302469A43BE
:100CA000104604220A401043014A106070470000B9
:100CB00000FA0140012806D10649096802221143C1
:100CC000044A116005E00349096802229143014A80
:100CD0001160704700FA01400148806880B2704797
:100CE00000FA014010B5012000F03CFC07F040F88C
:100CF000012007F04FF8022007F02AF8012007F042
:100D000015F80A20FFF784FF0120FFF76FFF04208A
:100D1000FFF7C0FF0120FFF7CDFF01208004FFF7A0
:100D200055FF0020FFF7A6FF044800F04DF8002013
:100D3000FFF77CFF0020FFF78BFF10BDFF070000CF
:100D400010B5012000F00EFC07F012F8012007F0AA
:100D500021F8022006F0FCFF012006F0E7FF052045
:100D6000FFF756FF0120FFF741FF0420FFF792FF36
:100D70000120FFF79FFF01208004FFF727FF0020DD
:100D8000FFF778FF044800F01FF80020FFF74EFF40
:100D90000020FFF75DFF10BDFF0700000548C06899
:100DA000FF2101310840002801D0012070470020B8
:100DB000FCE7000000FA0140FF2001300149C86053
:100DC0007047000000FA01404105490D014A516099
:100DD0007047000000FA014010B5012000F0C2FB8E
:100DE00006F0C6FF012006F0D5FF022006F0B0FF96
:100DF000012006F09BFF0F20FFF70AFF0120FFF7FD
:100E0000F5FE0420FFF746FF0120FFF753FF0748D8
:100E1000FFF7DAFF01208004FFF7D8FE0020FFF77C
:100E200005FF0020FFF714FF10BD0000FF070000C2
:100E300070B505460E4614462946204600F07CFB58
:100E4000044804600448066002F0EEFC02F00AFA6E
:100E500070BD0000340400203804002070B5054641
:100E60000E4614462946204600F066FB04480460FE
:100E70000448066002F0D8FC00F024FE70BD0000BB
:100E8000340400203804002010B50121074800F088
:100E9000B7FC022000F0D4F94021054800F0A7F982
:100EA00001224021024801F0AAFA10BD070000010A
:100EB000400D004030B50246002018E0002112E04D
:100EC000130184001B195B180A4CE35C84000A4D73
:100ED0002D686419645C63408400074D2D686419B3
:100EE00063544B1CD9B20429EADB431CD8B2042852
:100EF000E4DB30BDD817002034040020F8B50546E7
:100F00000E46002E22D02868002800D1F8BD2C689B
:100F100001E0274664686068002802D02088B0425B
:100F2000F7D12088B04210D109480078401E084906
:100F300008702868A04202D16068286001E06068FB
:100F40007860204608F08CF8002400BF00BFDDE781
:100F50002C04002010B50121794800F051FC00223A
:100F6000FF210131774805F087FD00228021754877
:100F7000403005F081FD002240217248403005F0EC
:100F80007BFD012291036F48803002F0EEF80122D0
:100F9000D1036C48803002F0E8F801225102694820
:100FA000403002F0E2F80022012109036548803850
:100FB00005F062FD00220121C9026248803805F077
:100FC0005BFD012109035F48803801F00CFA012123
:100FD000C9025C48803801F006FA00220121C903E9
:100FE0005848803805F048FD0121C903554880382C
:100FF00001F0F9F90022012189035248803805F0F7
:101000003BFD012189034F48803801F0ECF90022B3
:10101000012149034B48803805F02EFD0121490389
:101020004848803801F0DFF90021082002F0D8F8A4
:1010300000220221434802F098F800220121414891
:10104000C03805F019FD002202213E48C03805F0E5
:1010500013FD002204213B48C03805F00DFD00229D
:1010600008213848C03805F007FD00220121354825
:10107000803005F001FD01213248803001F0B5F9E2
:10108000002220212F4802F070F8002210212D4864
:1010900002F06BF8012204212A48803802F065F83A
:1010A000012208212748803802F05FF8012251030D
:1010B0002448C03802F059F800221021214880301D
:1010C00005F0DAFC002208211E48803005F0D4FC2F
:1010D000012211461B4802F048F80021012002F0CD
:1010E0007FF80022FF2101311648803805F0C4FC4A
:1010F0000022012149021348803805F0BDFC00227E
:1011000004211048C03005F0B7FC002208210D482A
:10111000C03005F0B1FC00220121490309484038E4
:1011200002F023F8002280210648C03002F01DF8AA
:10113000002220210348803002F017F810BD000083
:1011400007000001C00C00407FB506460D4614465E
:101150006A462946304601F071F80098A84227D126
:101160006846C079002823D1E007C00F002803D1CA
:101170006846407900281BD1E007C00F002803D043
:1011800068464079012813D102202040002803D16D
:101190006846807900280BD102202040002803D027
:1011A00068468079012803D16846007902281DD05D
:1011B000029500206946C873E007C00F002801D1DE
:1011C000487302E00120694648730220204000284D
:1011D00002D16946887302E00120694688730220C3
:1011E0006946087302A9304601F0BAF87FBD7FB5A1
:1011F00005460C466A462146284601F01FF800982D
:10120000A0420FD16846C07900280BD168464079CA
:10121000002807D168468079002803D16846007904
:1012200003280BD0029400216846C1734173817377
:101230000321017302A9284601F092F87FBD000046
:1012400070B505460024002600F080F9002802D180
:10125000012000F087F9002416E00120A040064696
:101260002846304000280ED00C4800680121A140DB
:1012700088430A490860084681686200032090405C
:10128000014306488160641C042CE6D300F05EF93B
:10129000012802D1002000F065F970BD00FC01407A
:1012A00000B587B0684600F069F90BA006F092FD22
:1012B00017A006F08FFD1EA220A123A006F08AFD34
:1012C0002AA0009906F086FD03A006F083FD0FA07A
:1012D00006F080FD07B000BD2F2A2A2A2A2A2A2AD2
:1012E0002A2A2A2A2A2A2A2A2A2A2A2A2A2A2A2A5E
:1012F0002A2A2A2A2A2A2A2A2A2A2A2A2A2A2A2A4E
:101300002A2A2A2A2A2A2A2A2A2A2A2F0D0A0000C9
:101310002F6170706C69636174696F6E566572736A
:10132000696F6E2073746172742F0D0A00000000E3
:1013300031313A33353A3433000000004A756E20BB
:1013400020372032303234004275696C64204461A9
:101350007465202020202020202020202020203DD7
:101360002025732025730D0A000000005379737443
:10137000656D20436C6F636B204672657175656E99
:1013800063793A20256C7520487A0A000149C862C1
:101390007047000000600140012806D10649096835
:1013A00080221143044A116005E003490968802244
:1013B0009143014A1160704700600140012806D145
:1013C0000649096801221143044A116005E00349F6
:1013D000096849084900014A1160704700600140EE
:1013E0000146064A1068082302469A43104608221E
:1013F0000A401043014A106070470000006001403D
:10140000012806D10649C96801221143044AD16066
:1014100005E00349C96849084900014AD16070479D
:101420000060014010B500F00DF8002806D0044817
:101430000068401C0249086000F010F810BD000070
:10144000B003002004480069C007C00F002801D085
:10145000012070470020FCE70060014001200149A5
:1014600008617047006001400149886270470000D0
:1014700000600140012904D1026880231A43026000
:1014800003E0026880239A430260704710B51D484C
:1014900000F042F8012809D11A4800F04AF819482A
:1014A00000F044F801201849487029E015484430FC
:1014B00000F032F8012823D11248443000F039F806
:1014C0001048443000F032F810480078401C0F49B2
:1014D000087005210D480078FEF726FE00290FD17F
:1014E00001200B4908700B480078401CC0B2094924
:1014F0000870032804DB002102484430FFF7BAFFDC
:1015000010BD0000003001403C0400200400002019
:10151000FA0000200A0100200146086C1022104049
:10152000002801D0012070470020FCE71021016451
:1015300070470821016470470246002003E00B5CFD
:101540001354431CD8B21028F9DB704704480068D4
:101550000007000F0A2801D1012070470020FCE796
:1015600000E00140012803D10A21034A116002E092
:101570000521014A1160704700E0014000B50246B4
:1015800000230020D060106110605060906000F077
:10159000A1F9012807D100F085F903461B0C581C5E
:1015A0003B494843D06000F05FF901280ED100F0BC
:1015B0006FF903461B0C581C36494843106100F074
:1015C0005FF9082802D110694000106100F0FAF9B3
:1015D000034600BF002B06D0012B07D0022B08D0FA
:1015E000032B0DD108E0D06810600CE02A48106091
:1015F00009E01069106006E00120C003106002E0FD
:10160000D068106000BF00BF00F098F903461B0AC5
:10161000042B06D0052B08D0062B0AD0072B10D19F
:101620000BE01068400850600EE0106880085060C1
:101630000AE01068C008506006E0106800095060B9
:1016400002E01068506000BF00BF00F08FF9034651
:101650001B0C042B06D0052B08D0062B0AD0072B19
:1016600010D10BE05068400890600EE05068800890
:1016700090600AE05068C008906006E05068000979
:10168000906002E05068906000BF00BF00BD0000A5
:1016900000127A0040420F00001BB700012806D15B
:1016A0000649896901221143044A916105E0034911
:1016B000896949084900014A916170470024004046
:1016C000704700000548C069FF210131084000282B
:1016D00001D0012070470020FCE7000000240040FA
:1016E00010B50446012C02D11148036813E0022C06
:1016F00003D10F484038C36B0DE0032C03D10C48D5
:101700004038836B07E0042C03D109484038436B11
:1017100001E007480368180CD94389B2884203D115
:10172000D8B200F0F5F802E06B2000F0F1F810BD3F
:1017300040FBFF1F012806D10749096B0202114334
:10174000054A116306E00449096BFF220132914307
:10175000014A116370470000002400400146054A19
:10176000106B800880008A07920F1043014A1063B3
:101770007047000000240040012806D10749096B8A
:1017800042021143054A116306E00449096B012234
:1017900052029143014A1163704700000024004047
:1017A0000146064A106B0C2302469A4310460C224F
:1017B0000A401043014A10637047000000240040B3
:1017C000012806D10649496B10221143044A51638E
:1017D00005E00349496B10229143014A5163704768
:1017E000002400400146054A506B800880008A07AB
:1017F000920F1043014A50637047000000240040DC
:1018000030B502460B4600200F2424061440FF2565
:101810002D066419002C09D06419002C08D0641915
:10182000002C08D06419002C0BD107E00D4809E00A
:101830000C48001D06E00B48083003E009480C3056
:1018400000E000BF00BF00280BD092B20121914000
:10185000002B03D004680C43046002E004688C434E
:10186000046030BD2024004004480069C007C00F58
:10187000002801D0012070470020FCE70024004030
:101880000248006908210840704700000024004019
:1018900002480069024908407047000000240040E7
:1018A0000000FF03024840680F2109040840704708
:1018B000002400400146064A50680F231B040246DC
:1018C0009A4310461A460A401043014A5060704736
:1018D0000024004004484068C007C00F002801D021
:1018E000012070470020FCE700240040012806D1B9
:1018F0000649496801221143044A516005E0034941
:10190000496849084900014A516070470024004075
:101910000146044A9068000A0002CAB21043014A14
:10192000906070470024004010B504462068FFF71F
:10193000C1FF2079FFF7DAFF10BD00000248006800
:101940000721090208407047002400400146064A6A
:10195000106807231B0202469A4310461A460A40A3
:101960001043014A1060704700240040024800689C
:101970000721090408407047002400400146064A38
:10198000106807231B0402469A4310461A460A4071
:101990001043014A1060704700240040012806D11E
:1019A0000749096842061143054A116006E00449E7
:1019B0000968012252069143014A116070470000F4
:1019C00000240040024800684007400F70470000B4
:1019D000002400400146054A1068C008C0004A07BC
:1019E000520F1043014A106070470000002400406D
:1019F00010B504462068FFF7EDFF6068FFF7A6FF0B
:101A0000A068FFF7BBFF207BFFF7C8FF10BD0000F9
:101A1000012806D10649496901221143044A51614E
:101A200005E00349496949084900014A5161704785
:101A3000002400400146064A506907231B02024663
:101A40009A4310461A460A401043014A50617047B3
:101A50000024004005480068012149020840002890
:101A600001D0012070470020FCE700000054014035
:101A700010B500F015F801280CD100F01DF8FFF7A3
:101A8000E9FF012803D104A006F0A4F902E003A0B5
:101A900006F0A0F910BD0000310D0A00320D0A0059
:101AA0000448C068C007C00F002801D0012070475B
:101AB0000020FCE70054014001200149C860704744
:101AC0000054014010B500240020FFF7F3F9012471
:101AD0000AE005F0E5FB05F07DFB04F0B7FE2046CB
:101AE000FFF7E8F9601CC4B20A2CF2DB05F0D8FB62
:101AF00005F070FB0A20FFF7DDF910BDF8B50446CC
:101B00000E4600250027FFF721FD002802D1012005
:101B1000FFF728FD002512E00120A84007463046C7
:101B2000384000280AD020680121A940884320605D
:101B3000A1686A00032090408143A1606D1C042DC0
:101B4000EAD3FFF703FD012802D10020FFF70AFDC9
:101B5000F8BD70B50A460021002300BF12E0012441
:101B60008C40234614461C40002C0AD004680125F2
:101B70008D40AC430460C4684E000325B540AC43BF
:101B8000C460491C1029EAD370BD032001218907D4
:101B9000486070470146064AD069131502469A43C9
:101BA00010461A460A401043014AD06170470000AF
:101BB00040040040012806D10649C96901221143A9
:101BC000044AD16105E00349C96949084900014A4D
:101BD000D1617047400400400146064AD069931520
:101BE00002469A4310461A460A401043014AD06101
:101BF0007047000040040040012806D10649C96929
:101C000004221143044AD16105E00349C969042251
:101C10009143014AD161704740040040012806D138
:101C20000649C96902221143044AD16105E003490A
:101C3000C96902229143014AD161704740040040C2
:101C40000146064AD06903231B0302469A43104605
:101C50001A460A401043014AD061704740040040D0
:101C60000146064AD069531502469A4310461A4661
:101C70000A401043014AD061704700004004004010
:101C80000004054AD169054A1140D243024011437C
:101C9000014AD1617047000040040040FFFF00E0AE
:101CA000C103490C014A1162704700004004004022
:101CB00030B50246D400064D631918683025044635
:101CC000AC43204630240C402043186030BD000057
:101CD000040400400146C800054BC21804231068E4
:101CE0001840002801D0012070470020FCE70000C8
:101CF0000404004010B50246D300074C181901290E
:101D000004D1042403682343036003E0042403682C
:101D1000A343036010BD00000404004010B5024658
:101D2000D300074C1819012904D102240368234366
:101D3000036003E002240368A343036010BD0000B6
:101D40000404004030B50246D400064D63191868FB
:101D5000ED140446AC4320462C460C40204318604A
:101D600030BD00000404004030B50246D400064DEA
:101D70006319186803252D030446AC4320462C46FE
:101D80000C402043186030BD0404004030B50246CA
:101D9000D400064D6319186807252D020446AC438C
:101DA00020462C460C402043186030BD04040040FF
:101DB00030B50246D400054D631909041868044C77
:101DC0002040E4430C402043186030BD0404004030
:101DD000FFFF00E010B50246D300074C1819012997
:101DE00004D1082403682343036003E00824036844
:101DF000A343036010BD00000404004010B5024678
:101E0000D300074C1819012904D101240368234386
:101E1000036003E003685B085B00036010BD000023
:101E20000404004030B50246D400064D631918681A
:101E300040250446AC43204640240C402043186013
:101E400030BD0000040400400146C800014BC21828
:101E5000106870470804004010B5C300014C1A19FF
:101E6000116010BD08040040012806D10649096828
:101E700001221143044A116005E003490968490839
:101E80004900014A116070470004004010B503206A
:101E9000FFF720FF012807D1032000F007F80128F1
:101EA00002D1032000F012F810BD000001460648E0
:101EB000806A012212048A401040002801D00120CB
:101EC00070470020FCE700004004004001210904A5
:101ED0008140014A916270474004004010B50446B9
:101EE00020780B2823D120780021FFF787FF606836
:101EF000FFF7C6FEA068FFF7A3FE6069FFF74AFE82
:101F0000606AFFF7ADFEA06AFFF766FE607FFFF72D
:101F100073FEA07FFFF782FE2078216AFFF79CFF07
:101F2000E06AFFF7BDFEE07FFFF744FE2FE0207878
:101F30000021FFF763FF20786168FFF739FF207801
:101F4000A168FFF711FF2078E168FFF7FBFE20781A
:101F50002169FFF71BFF20786169FFF763FF207895
:101F6000A169FFF7A5FE217F2078FFF733FF617F8E
:101F70002078FFF7BFFEA17F2078FFF7CFFE207803
:101F8000216AFFF769FFE17F2078FFF737FF10BD77
:101F9000F7B582B006460F463D460498019000BF53
:101FA0004021174800F01FFA01218903144800F06E
:101FB0001CFA00BF032005F059F92902080E05F0AC
:101FC00055F92904080E05F051F9E8B205F04EF96B
:101FD000002405E0FF2005F049F93055601C84B26B
:101FE00001988442F6DB00BF4021054800F0FDF96E
:101FF00001218903024800F0F8F900BF05B0F0BDE7
:10200000800C00400146054A1068800880008A075D
:10201000920F1043014A106070470000001000400A
:1020200070B505462C4600BF4021144800F0DBF98E
:1020300001218903114800F0D8F900BF032005F001
:1020400015F92102080E05F011F92104080E05F01A
:102050000DF9E0B205F00AF9FF2005F007F9064690
:1020600000BF4021054800F0C0F901218903034861
:1020700000F0BBF900BF304670BD0000800C00408E
:102080001CB504462046FFF7CBFF69460870601C6C
:10209000FFF7C6FF014668464170A01CFFF7C0FF6E
:1020A000014668468170E01CFFF7BAFF01466846AA
:1020B000C170201DFFF7B4FF014668460171601D25
:1020C000FFF7AEFF014668464171A01DFFF7A8FF6C
:1020D000014668468171E01DFFF7A2FF0146684690
:1020E000C1710078FF2820D168464078FF281CD1B4
:1020F00068468078FF2818D16846C078FF2814D138
:1021000068460079FF2810D168464079FF280CD135
:1021100068468079FF2808D16846C079FF2804D135
:102120006A4600200146FEF7A3F86846FEF789F8E4
:102130001CBD38B504462046FFF772FF694608709B
:10214000601CFFF76DFF014668464170A01CFFF759
:1021500067FF014668468170E01CFFF761FF694632
:10216000C870009838BD38B504462046FFF758FFC0
:1021700069460870601CFFF753FF014668464170CE
:10218000A01CFFF74DFF014668468170E01CFFF779
:1021900047FF6946C870009838BD00003EB5044648
:1021A0000422214602A8FFF7F3FE642006F096FE03
:1021B0000422214601A8FFF7EBFE0199029888420C
:1021C0000AD11D490298884201D802983EBD0020DC
:1021D000C04302900298F9E7642006F07FFE0422D3
:1021E00021466846FFF7D4FE01990298884203D041
:1021F0000099029888420AD10F490298884201D872
:102200000298E3E70020C04302900298DEE70099BD
:10221000019888420AD108490198884201D801985A
:10222000D4E70020C04301900198CFE70020C043CD
:1022300001900198CAE7000000E9A435F0B5044612
:102240000025002307E001269E400E403546002D64
:1022500000D002E05B1C102BF5D300BF102B36D250
:102260001D46116026680E403046E840012802D124
:102270000126D67101E00026D67166680E40EE4058
:102280003046012801D1967101E000269671A668BA
:102290000E40EE403046012801D1567101E0002683
:1022A0005671E6686F00FE40B007800F002802D12B
:1022B000002616710BE0012802D10126167106E0F6
:1022C000022802D10226167101E003261671F0BD24
:1022D00010B501211A48FFF793FA1A491A48FFF777
:1022E00038FC1A4918484030FFF733FC18491648A3
:1022F0008030FFF72EFCFF2134311348C030FFF748
:1023000028FC132149011348FFF723FC1249114807
:102310004030FFF71EFC0C210E488030FFF719FCFF
:1023200009210E48FFF7EAFB002101208006FFF794
:1023300067FA0020FFF744FA002005F0F7FC10BD13
:10234000070000010F200000000C00400CBB000043
:1023500040600000000D004019C0000000FC01407A
:10236000F0B502460B4600210024002500BF2DE0F9
:1023700001268E4034461E6826403546A54224D1AB
:1023800010680646A6433046DE798E403043106022
:1023900050680646A64330469E798E4030435060D2
:1023A00090680646A64330465E798E403043906082
:1023B0004F000326BE403446D0680646A64330464A
:1023C0001E794F00BE403043D060491C1029CFD346
:1023D000F0BD02460020D3690B40002B01D0012044
:1023E00000E00020704781617047416170470269D9
:1023F0000A40002A01D0816100E04161704710B5B8
:102400001346826A012B03D114460C43224602E094
:1024100014468C432246826210BD000070B5002530
:102420000020674948706749087000F00BFE664855
:1024300000786649097840186549087008460078B0
:10244000624908700020604908706148007864287B
:1024500002DD01205E4908705E4800685C49097829
:10246000884209D25B4800685B494018584909789E
:10247000401A5A49086006E05648006854490978ED
:10248000401A5649086000F0D3FB05204C4988707B
:10249000122088715248017B494823300171090A92
:1024A000417101204F4988750020C8754448233088
:1024B00041790279080210431E2807DB4048233087
:1024C0004179027908021043FF2805DD5A213C4872
:1024D000233001710021417100255CE000F0B2FD64
:1024E0000A2006F0D3FC6D1C35488078002809D0FE
:1024F00033488078032805D131484078002801D03E
:1025000000F0F6FB2E488078002803D02C4988790B
:1025100004F072F92A482330417902790802104305
:10252000002802D03048854235D330A000F068F84A
:1025300000F088FDC82006F0A9FC1920400106F033
:10254000A5FCC82006F0A2FC1920400106F09EFC64
:102550000020284908701B49087001212148817515
:102560000021C1752448C07C401CC1B22248C174FE
:1025700020380078002805DD1F48807C401CC1B24F
:102580001D48817400211D48C17201730C48203020
:10259000417200F057FD0B48007800289ED10024BE
:1025A0000AE000F04FFDC82006F070FC1920400141
:1025B00006F06CFC601C84B2142CF2DB70BD0000D1
:1025C000781D0020020600200E0600200F060020C5
:1025D0001006002014060020EE020000DC0500209A
:1025E0000C1A0020A31D002050C300004154434C8E
:1025F0004F53450004060020811A0020671D00206B
:1026000070B504462046FDF70BFEC6B2002505E076
:10261000207807F0BBF9641C681CC5B2B542F7DB33
:10262000012006F033FC70BD70B5002400250120A8
:10263000FEF70EFBFEF7C0FB06F004F9002803D1FD
:10264000FEF74AFB054601E0002070BD284606F073
:1026500075F804462046F8E738B5002000900024BD
:102660000120FEF7F5FAFEF7A7FB06F0EBF80028CD
:1026700003D1FEF731FB044601E0002038BD2046BF
:1026800006F0AEF800900098F8E70000F0B587B0CB
:102690000026FEF727FB10211F48FFF7A6FE132098
:1026A00007F098F9041E30D0082161700021A17054
:1026B0000A202070204600F04BFA07463846FEF705
:1026C00058F80190FEF70EF9144A154B0391029049
:1026D000FDF764FF05910490FEF740F90546284692
:1026E000FEF700F90F4A104B03910290FDF756FFD9
:1026F00005910490FEF732F9064610210648FFF7CF
:1027000072FE204606F0ACFC00240020FEF7A0FA82
:10271000304607B0F0BD0000400D0040FCA9F1D2EA
:102720004D62503F9A99999999990540F0B587B0B3
:102730000026FEF705FB08211F48FFF756FE142070
:1027400007F048F9041E30D0082161700021A17003
:1027500005202070204600F0FBF907463846FEF7BA
:1027600008F80190FEF7BEF8144A154B0391029049
:10277000FDF714FF05910490FEF7F0F80546284692
:10278000FEF7B0F80F4A104B03910290FDF706FFD9
:1027900005910490FEF7E2F8064608210648FFF787
:1027A00022FE204606F05CFC00240020FEF750FAD2
:1027B000304607B0F0BD0000400D0040FCA9F1D24A
:1027C0004D62503F9A9999999999094070B5FEF7D1
:1027D00003FB132007F0FEF8041E0AD008216170E5
:1027E0000021A170FFF720FF0546204606F038FCC7
:1027F00000240020FEF72CFA284670BDF0B585B005
:1028000006460127002523E002A804F051FB684694
:1028100004F04EFB002408E002A8005D6946095D53
:10282000884200D003E0601CC4B2072CF4DB00BF78
:10283000072C0BD10027072202A93046FDF7B8FC70
:10284000072202A90548FDF7B3FC03E0681CC5B2E6
:10285000032DD9DB00BF384605B0F0BDA004002031
:102860000EB50722AA49002004F01EFAA8480078F5
:10287000F0210840002819DBA548007808405028BE
:1028800014DCA34800780007000F00280ADBA048EA
:1028900000780007000F092804DC9D4800789D4956
:1028A000887006E000209B49887002E0002099496A
:1028B000887097484078F0210840002819DB944838
:1028C00040780840502814DC914840780007000FF9
:1028D00000280ADB8E4840780007000F092804DC36
:1028E0008B4840788B49487006E000208949487041
:1028F00002E000208749487085488078F021084030
:1029000000110A214843824989780907090F4018B4
:10291000182823DA7E488078F0210840002819DB47
:102920007B4880780840202814DC794880780007AC
:10293000000F00280ADB764880780007000F09287E
:1029400004DC73488078734908700AE000207149FC
:10295000087006E000206F49087002E000206D4911
:1029600008706B48C0786B49487169480079F0215C
:10297000084000110A214843654909790907090FF0
:102980004018202831DA62480079F021084000110F
:102990000A2148435E4909790907090F40180028B0
:1029A00023DD5B480079F0210840002819DB5848F6
:1029B00000790840302814DC554800790007000FE2
:1029C00000280ADB524800790007000F092804DCC0
:1029D0004F4800794F4908710AE001204D490871BC
:1029E00006E001204B49087102E0012049490871C5
:1029F00047484079F021084000110A2148434449E2
:102A000049790907090F40180D2831DA4048407903
:102A1000F021084000110A2148433D49497909073E
:102A2000090F4018002823DD39484079F02108407B
:102A3000002819DB364840790840102814DC344857
:102A400040790007000F00280ADB31484079000771
:102A5000000F092804DC2E4840792E49C8700AE08E
:102A600012202C49C87006E012202A49C87002E0E2
:102A700012202849C87026488079F02108400011AA
:102A80000A214843224989790907090F4018642817
:102A900026DA1F488079F021084000281CDB1C48FA
:102AA00080790840902817DC194880790007000FCA
:102AB00000280DDB164880790007000F092807DC85
:102AC000134880790121490340181249C8800AE05F
:102AD00011481049C88006E00F480E49C88002E03E
:102AE0000D480C49C880642006F0D0F90948807868
:102AF00008494978074A12780092019102900548E6
:102B00000379C278C18805A005F064F90EBD000004
:102B1000F22300201A0600201520000045585445D5
:102B2000524E414C205254432054494D45203D20A3
:102B300025582D253032582D253032582D2530324C
:102B4000582D253032582D25303258200D0A0000DE
:102B5000FEB5044600200090002509E0FFF77CFD4B
:102B60000746AA00E01C11183846FDF778FB6D1CDB
:102B7000A178627808021043A842EFD800252EE021
:102B80006E1C25E0B200E11C5018FDF750FB074613
:102B9000AA00E11C5018FDF74AFB874217D2B20089
:102BA000E11C5018FDF743FB0190AA00E11C5018EE
:102BB000FDF73DFB0746B200E01C11183846FDF753
:102BC0004EFBAA00E01C11180198FDF748FB761C8B
:102BD000A178627808021043B042D3D86D1CA17866
:102BE000627808021043A842CAD8012002900BE084
:102BF00002998A00E11C5018FDF719FB0099401852
:102C000000900298401C0290A1786278080210435C
:102C1000401E02998842EBD8A278637810021843CC
:102C2000811E0098FDF76AFA00900098FEBD000032
:102C300010B588B020216846FDF7D3FA1A216846FE
:102C400001704170002405E00021A01C6A46115467
:102C5000601CC4B2082CF7DB2720224908706C20C6
:102C60004870512088706920C870AA216846817315
:102C70002621C173002407E01A48015D20460A306E
:102C80006A461154601CC4B2042CF5DB1648017B63
:102C90006846017400214174002406E000212046AA
:102CA00012306A461154601CC4B2072CF6DB0020B7
:102CB00069464876002409E06846407E6946095D19
:102CC0004018C1B268464176601CC4B2192CF3DBCF
:102CD0001620694688761E22044804F0A3FF08B037
:102CE00010BD0000FA0500200C1A00200068014009
:102CF00010B58448407A00287ED1FFF7B1FD8248A4
:102D00008079824948738048C07888737E4800790A
:102D1000C8737D48007808747B48407848747A48C6
:102D2000807888747A480078002865DD78480078D3
:102D300078490870084600787749087004E07648BA
:102D40000078001F74490870734800780428F6DC86
:102D50007148007804280AD16E490878C117890F94
:102D600009188910694A1176090A51760AE06949F9
:102D70000878C117890F09188910491C634A117610
:102D8000090A517685206149887264480875000AED
:102D900048755C482038C079C876614801785B483E
:102DA000203081745F48C17C5848203001755C48F0
:102DB000817956482030C1745749097850225143CF
:102DC00008461F30C117090F091809110901411AD6
:102DD000554A1170504909785022514308461F3016
:102DE000C117090F09180905090E504A1170474902
:102DF000487E097E000200E055E00843012853DDCB
:102E00004249C87D897D00020843404A517E127EB6
:102E10000902114388421ADA04213C4820304176E5
:102E20002038807E80210840002806D1FF216E31A5
:102E30003648C172090A017305E0FF216F3133483A
:102E4000C172090A0173002006F004FC58E02F4902
:102E5000C87D897D000208432C4A517E127E0902FA
:102E6000114388424CD12C480178284820304176C3
:102E70002038807E80210840002809D1264800782B
:102E8000502148432D302149C872000A087307E0D9
:102E90002648007800011E301C49C872000A0873D9
:102EA000012006F0D7FB2BE01849487E097E00027E
:102EB0000843012824D10121144881750021C175DE
:102EC000154801781148203041762038807E8021D5
:102ED0000840002809D110480078502148432D307F
:102EE0000A49C872000A087307E010480078000118
:102EF0001E300649C872000A0873012006F0AAFBBA
:102F000010BD0000981D00201A060020A31D0020FF
:102F100010060020EC050020ED0500206084000074
:102F20002C1A00200C1A002030040020310400204C
:102F300070B500260320FEF787FF05461C48854232
:102F400016D0022005F0A2FF0CE00320FEF77CFF64
:102F50000546022005F09AFF3046711C8EB26428A7
:102F600000DD04E00320FEF76FFFA842EDD101E091
:102F7000012070BD0E48281A84B2002C15D00D48CF
:102F8000C4730320FEF7A2FF00210320FEF736FFE3
:102F900007490320FEF760FF01210320FEF72EFF03
:102FA0000121044801740020E3E70120E1E700006B
:102FB000671B0020671D002070B500260520FEF766
:102FC00043FF05461D48854216D0022005F05EFFEE
:102FD0000CE00520FEF738FF0546022005F056FFFD
:102FE0003046711C8EB2642800DD04E00520FEF737
:102FF0002BFFA842EDD101E0012070BD0F48281A37
:1030000084B2002C17D00E480470210A41700520AC
:10301000FEF75CFF00210520FEF7F0FE07490520C2
:10302000FEF71AFF01210520FEF7E8FE0120044902
:1030300088700020E1E70120DFE70000480600205B
:10304000480A002001480249086070475A5A341261
:103050000014014010B501210448FEF7D1FB062001
:1030600003494860FFF7EEFF10BD000005000001B6
:103070000014014010B501210648FEF7C1FB0022F3
:103080000821054803F0F8FC00220421024803F05F
:10309000F3FC10BD07000001C00C00401CB500206F
:1030A00000900120694608716846FEF73DFC01204A
:1030B000FEF716FB1CBD00000A2005490860054804
:1030C000008CC0B20449C8610520014908607047FE
:1030D00000E0014000FBFF1F00F801401FB5002485
:1030E00001211948FEF78CFB02211848FEF77FF8F2
:1030F00004211648FEF77BF80120FEF789FC072023
:103100000002FEF797FC052005F0C0FE0120FEF747
:10311000C5FA05E019200002844200D304E0641CD3
:10312000FEF7D0FA0028F5D000BF01200090002063
:10313000019002900120694608736846FEF758FC2A
:10314000034805F07FFE1FBD07000001400D004051
:10315000001BB70010B50020FEF754FFFFF79EFFDD
:10316000FFF7AAFFFFF7BAFF10BD7FB506460D4671
:1031700014466A4629463046FFF760F80098A84290
:1031800017D16846C079012813D1684640790128D3
:103190000FD1002C03D168468079002809D1012C79
:1031A00003D168468079012803D168460079002858
:1031B00014D0029501216846C1734173002C03D1DC
:1031C00000206946887302E0012069468873002068
:1031D0006946087302A93046FFF7C2F87FBD0000B8
:1031E000F8B505460E4600240027FEF7AFF9002883
:1031F00002D10120FEF7B6F9002426E00120A0400C
:1032000007462846384000281ED0002E07D1144813
:1032100040680121A14088431149486006E01048F8
:1032200040680121A14008430D4948600C4881686D
:1032300062000320904081430948816000680121B9
:10324000A140084306490860641C042CD6D3FEF74D
:103250007DF9012802D10020FEF784F9F8BD0000B5
:1032600000FC014010B500240A20FDF723FE0924CC
:103270000AE000F071FA00F0BBFA2046FDF71AFEF2
:1032800000F00CF8601EC4B2002CF2DC00F064FA0E
:1032900000F0AEFA0020FDF70DFE10BD30B589B08C
:1032A000002008904FE208988000FE490968085CF9
:1032B000079008988000FB490968401840780690FC
:1032C00008988100F74800680818807805900898E9
:1032D0008000F44909684018C0780490079806F007
:1032E000E5FE0446079806F0E1FE039006F0DEFED8
:1032F0004440079806F0DAFE029006F0D7FE0390ED
:1033000006F0D4FE4440079806F0D0FE019006F087
:10331000CDFE029006F0CAFE039006F0C7FE0698A6
:1033200006F0C4FE05460698454006F0BFFE039031
:1033300006F0BCFE069806F0B9FE029006F0B6FE56
:10334000039006F0B3FE4540069806F0AFFE0190EC
:1033500006F0ACFE029006F0A9FE039006F0A6FE71
:103360006C40059806F0A2FE0598054606F09EFE04
:10337000039006F09BFE4540059806F097FE0290EC
:1033800006F094FE039006F091FE4540059806F085
:103390008DFE019006F08AFE029006F087FE0390F3
:1033A00006F084FE6C40049806F080FE0498054602
:1033B00006F07CFE039006F079FE049806F076FE97
:1033C000029006F073FE039006F070FE45400498EC
:1033D00006F06CFE019006F069FE029006F066FEB3
:1033E000039006F063FE6C4008988000AD490968C0
:1033F0000C54079806F05AFE0798044606F056FE4D
:10340000039006F053FE079806F050FE029006F077
:103410004DFE039006F04AFE4440079806F046FE33
:10342000019006F043FE029006F040FE039006F085
:103430003DFE069806F03AFE0546069806F036FE72
:10344000039006F033FE4540069806F02FFE0290EA
:1034500006F02CFE039006F029FE4540069806F083
:1034600025FE019006F022FE029006F01FFE03905A
:1034700006F01CFE6C40059806F018FE05460598FF
:10348000454006F013FE039006F010FE059806F086
:103490000DFE029006F00AFE039006F007FE45407E
:1034A000059806F003FE019006F000FE029006F07B
:1034B000FDFD039006F0FAFD6C40049806F0F6FD61
:1034C0000498054606F0F2FD039006F0EFFD454036
:1034D000049806F0EBFD029006F0E8FD039006F07C
:1034E000E5FD4540049806F0E1FD019006F0DEFDA3
:1034F000029006F0DBFD039006F0D8FD6C400898C2
:1035000080006849096840184470079806F0CEFDAD
:103510000798044606F0CAFD039006F0C7FD444034
:10352000079806F0C3FD029006F0C0FD039006F078
:10353000BDFD4440079806F0B9FD019006F0B6FDC8
:10354000029006F0B3FD039006F0B0FD069806F079
:10355000ADFD0698054606F0A9FD039006F0A6FD10
:10356000069806F0A3FD029006F0A0FD039006F079
:103570009DFD4540069806F099FD019006F096FDE8
:10358000029006F093FD039006F090FD6C400598C4
:1035900006F08CFD0546059806F088FD039006F0C0
:1035A00085FD4540059806F081FD029006F07EFD00
:1035B000039006F07BFD4540059806F077FD0190ED
:1035C00006F074FD029006F071FD039006F06EFDAA
:1035D0006C40049806F06AFD05460498454006F0E4
:1035E00065FD039006F062FD049806F05FFD029011
:1035F00006F05CFD039006F059FD4540049806F086
:1036000055FD019006F052FD029006F04FFD03902B
:1036100006F04CFD6C4008988000224A1268801821
:103620008470079806F042FD04460798444006F06F
:103630003DFD039006F03AFD079806F037FD029035
:1036400006F034FD039006F031FD4440079806F083
:103650002DFD019006F02AFD029006F027FD039053
:1036600006F024FD069806F021FD0698054606F0B2
:103670001DFD039006F01AFD4540069806F016FD64
:10368000029006F013FD039006F010FD45400698E9
:1036900006F00CFD019006F009FD029006F006FD13
:1036A000039001E03404002006F000FD6C40059812
:1036B00006F0FCFC0598054606F0F8FC039006F0C1
:1036C000F5FC059806F0F2FC029006F0EFFC039082
:1036D00006F0ECFC4540059806F0E8FC019006F089
:1036E000E5FC029006F0E2FC039006F0DFFC6C4083
:1036F000049806F0DBFC0546049806F0D7FC03901E
:1037000006F0D4FC4540049806F0D0FC029006F088
:10371000CDFC039006F0CAFC4540049806F0C6FCB8
:10372000019006F0C3FC029006F0C0FC039006F086
:10373000BDFC6C4008988000064A12688018C4706E
:103740000898401C08900898042800DAABE509B0F6
:1037500030BD00003404002024490968487B234917
:1037600009684A7A214909684A73204909684A79EF
:103770001E4909684A721D4909684A781B49096847
:103780004A711A49096848701849096888781749C0
:103790000968897A154A1268917014490968887213
:1037A000124909688879114909688A7B0F490968B3
:1037B0008A710E49096888730C490968C8780B49F1
:1037C0000968C979094A1268D17008490968CA7A32
:1037D00006490968CA7105490968CA7B034909682D
:1037E000CA7202490968C873704700003404002097
:1037F00070B5002413E000250DE0A900094A126805
:103800008918085D05F056FCA900064A1268891857
:103810000855681CC5B2042DEFDB601CC4B2042C33
:10382000E9DB70BD34040020F8B500241FE0A000DF
:1038300043490968095CA000424A1154A000401C99
:103840003F490968095CA000401C1154A000801C7D
:103850003B490968095CA000801C1154A000C01CF1
:1038600037490968095CA000C01C1154641C042C71
:10387000DDD362E0002507E0601E80004019314979
:10388000085C694648556D1C042DF5D3A007800FD0
:10389000002825D16846067841780170817841700A
:1038A000C1788170C6706946087805F009FC6946E0
:1038B0000870487805F004FC69464870887805F07F
:1038C000FFFB69468870C87805F0FAFB6946C87046
:1038D0000878A1081C4A515C48406946087000E01D
:1038E00000BF201F80001749085C694609784840DE
:1038F000A100144A5054201F8000401C1146095C4E
:10390000684640784840A100491C5054201F800060
:10391000801C1146095C684680784840A100891CDB
:103920005054201F8000C01C1146085C6946C978AD
:103930004840A100C91C5054641C2C2C9AD3F8BDDB
:1039400038040020D8170020BEA2000010B5FF20C8
:10395000153002F001FCFF20163002F0FDFBFF20C5
:103960000F3002F0F9FBFF20103002F0F5FBFF20D2
:10397000183002F0F1FBFF20173002F0EDFBFF20C2
:103980000E3002F0E9FBFF200D3002F0E5FB0520D0
:1039900002F0E2FB062002F0DFFB072002F0DCFB76
:1039A000042002F0D9FB572002F0D6FB3F2002F0A2
:1039B000D3FB472002F0D0FB462002F0CDFB452090
:1039C00002F0CAFB4D2002F0C7FB4E2002F0C4FB00
:1039D0004F2002F0C1FB502002F0BEFB492002F054
:1039E000BBFB4A2002F0B8FB402002F0B5FB4220AE
:1039F00002F0B2FB4B2002F0AFFB482002F0ACFB20
:103A0000412002F0A9FB3C2002F0A6FB442002F07A
:103A1000A3FB4C2002F0A0FB432002F09DFB022000
:103A200002F09AFB032002F097FB012002F094FBC6
:103A3000002002F091FBFF20143002F08DFBFF20EC
:103A4000133002F089FBFF20123002F085FBFF20CB
:103A50000B3002F081FBFF200C3002F07DFBFF20D9
:103A6000053002F079FBFF20113002F075FBFF20DA
:103A70000A3002F071FBFF20093002F06DFB8B2051
:103A800002F06AFB822002F067FB832002F064FBF5
:103A90008C2002F061FB812002F05EFB802002F0AE
:103AA0005BFB8E2002F058FB872002F055FB86203E
:103AB00002F052FB852002F04FFB842002F04CFB09
:103AC000132002F049FB182002F046FBFF200330D0
:103AD00002F042FBFF20013002F03EFBF22002F038
:103AE0003BFBF02002F038FBE32002F035FBE02046
:103AF00002F032FBD32002F02FFBC82002F02CFB97
:103B0000BA2002F029FBB82002F026FBAA2002F01E
:103B100023FBA82002F020FB9B2002F01DFB982035
:103B200002F01AFBF52002F017FBF72002F014FB5D
:103B3000E52002F011FBE72002F00EFBD42002F09A
:103B40000BFBD72002F008FBC42002F005FBBF20CE
:103B500002F002FBAD2002F0FFFAAF2002F0FCFA07
:103B60009D2002F0F9FA9F2002F0F6FA08210120C8
:103B700000F079F80821022000F075F808210320F0
:103B800000F071F80821042000F06DF808210520EC
:103B900000F069F80821062000F065F808210720E8
:103BA00000F061F80821084600F05DF808210920BE
:103BB00000F059F808210A2000F055F808210B20E0
:103BC00000F051F808210C2000F04DF808210D20DC
:103BD00000F049F808210E2000F045F808210F20D8
:103BE00000F041F80821102000F03DF808211120D4
:103BF00000F039F80821122000F035F808211320D0
:103C000000F031F80821142000F02DF8014802F0EE
:103C1000BFFA10BDC822002030B50146C3175B0FA4
:103C20005B18DB10094CE35C0246C417640FA41850
:103C3000E410E400051B0124AC40A343C417640F47
:103C40006418E410014D2B5530BD0000C82200203F
:103C500000B58DB0302101A8FCF7C3FA01A802F02D
:103C600097FA0DB000BD70B505460C46152D01D371
:103C700002F06FFA6B007B449B885B009F446912E3
:103C80001400FC00E401CC02B4039C04840581060A
:103C9000690751083909210A090BF10BF90CE10DEB
:103CA000C90EB10F99108111230004F0CEF80A0655
:103CB0001C32485E748AA0B6CCE20F2002F04CFAA7
:103CC000172002F049FA152002F046FA0C2002F003
:103CD00043FA0D2002F040FA0E2002F03DFA1620C1
:103CE000FFF79AFFC6E00F20FFF796FF172002F0BC
:103CF00033FA152002F030FA0C20FFF78DFF0D206B
:103D0000FFF78AFF0E20FFF787FF1620FFF784FFDB
:103D1000B0E00F2002F020FA172002F01DFA152063
:103D2000FFF77AFF0C2002F017FA0D2002F014FAC8
:103D30000E20FFF771FF162002F00EFA9AE00F2016
:103D400002F00AFA172002F007FA152002F004FA2E
:103D50000C2002F001FA0D20FFF75EFF0E20FFF7A6
:103D60005BFF162002F0F8F984E00F20FFF754FF04
:103D7000172002F0F1F9152002F0EEF90C20FFF700
:103D80004BFF0D20FFF748FF0E2002F0E5F916204B
:103D900002F0E2F96EE00F2002F0DEF91720FFF7E3
:103DA0003BFF152002F0D8F90C2002F0D5F90D20C8
:103DB000FFF732FF0E2002F0CFF9162002F0CCF907
:103DC00058E00F2002F0C8F91720FFF725FF152053
:103DD00002F0C2F90C2002F0BFF90D2002F0BCF98C
:103DE0000E2002F0B9F9162002F0B6F942E00F20D9
:103DF00002F0B2F9172002F0AFF9152002F0ACF989
:103E00000C20FFF709FF0D20FFF706FF0E20FFF73C
:103E100003FF1620FFF700FF2CE00F2002F09CF9B3
:103E2000172002F099F9152002F096F90C2002F003
:103E300093F90D2002F090F90E2002F08DF9162072
:103E400002F08AF916E00F2002F086F9172002F03E
:103E500083F9152002F080F90C2002F07DF90D2085
:103E6000FFF7DAFE0E2002F077F9162002F074F95F
:103E700000E000BF00BFFBE6230003F0E6FF0A06F8
:103E80001C32485E748AA0B6CCE21F2002F064F9AE
:103E90003E2002F061F93D2002F05EF91C2002F0A4
:103EA0005BF9142002F058F91E2002F055F91D208C
:103EB000FFF7B2FEC6E01F20FFF7AEFE3E2002F085
:103EC0004BF93D2002F048F91C20FFF7A5FE142015
:103ED000FFF7A2FE1E20FFF79FFE1D20FFF79CFEAE
:103EE000B0E01F2002F038F93E2002F035F93D2005
:103EF000FFF792FE1C2002F02FF9142002F02CF99B
:103F00001E20FFF789FE1D2002F026F99AE01F20EF
:103F100002F022F93E2002F01FF93D2002F01CF9C8
:103F20001C2002F019F91420FFF776FE1E20FFF77F
:103F300073FE1D2002F010F984E01F20FFF76CFED5
:103F40003E2002F009F93D2002F006F91C20FFF79F
:103F500063FE1420FFF760FE1E2002F0FDF81D2016
:103F600002F0FAF86EE01F2002F0F6F83E20FFF7AC
:103F700053FE3D2002F0F0F81C2002F0EDF8142072
:103F8000FFF74AFE1E2002F0E7F81D2002F0E4F8D9
:103F900058E01F2002F0E0F83E20FFF73DFE3D20F4
:103FA00002F0DAF81C2002F0D7F8142002F0D4F85E
:103FB0001E2002F0D1F81D2002F0CEF842E01F20B2
:103FC00002F0CAF83E2002F0C7F83D2002F0C4F823
:103FD0001C20FFF721FE1420FFF71EFE1E20FFF716
:103FE0001BFE1D20FFF718FE2CE01F2002F0B4F886
:103FF0003E2002F0B1F83D2002F0AEF81C2002F0A5
:10400000ABF8142002F0A8F81E2002F0A5F81D203D
:1040100002F0A2F816E01F2002F09EF83E2002F007
:104020009BF83D2002F098F81C2002F095F814202F
:10403000FFF7F2FD1E2002F08FF81D2002F08CF831
:1040400000E000BF00BF13E6230003F0FEFE0A06F7
:104050001C32485E748AA0B6CCE25F2002F07CF885
:104060005E2002F079F85D2002F076F85C2002F024
:1040700073F8542002F070F8562002F06DF85520C5
:10408000FFF7CAFDC6E05F20FFF7C6FD5E2002F025
:1040900063F85D2002F060F85C20FFF7BDFD54205E
:1040A000FFF7BAFD5620FFF7B7FD5520FFF7B4FD27
:1040B000B0E05F2002F050F85E2002F04DF85D2085
:1040C000FFF7AAFD5C2002F047F8542002F044F804
:1040D0005620FFF7A1FD552002F03EF89AE05F2040
:1040E00002F03AF85E2002F037F85D2002F034F872
:1040F0005C2002F031F85420FFF78EFD5620FFF7C8
:104100008BFD552002F028F884E05F20FFF784FD46
:104110005E2002F021F85D2002F01EF85C20FFF71F
:104120007BFD5420FFF778FD562002F015F855204E
:1041300002F012F86EE05F2002F00EF85E20FFF74A
:104140006BFD5D2002F008F85C2002F005F85420B9
:10415000FFF762FD562001F0FFFF552001F0FCFF44
:1041600058E05F2001F0F8FF5E20FFF755FD5D206D
:1041700001F0F2FF5C2001F0EFFF542001F0ECFFB2
:10418000562001F0E9FF552001F0E6FF42E05F20F4
:1041900001F0E2FF5E2001F0DFFF5D2001F0DCFFB7
:1041A0005C20FFF739FD5420FFF736FD5620FFF75E
:1041B00033FD5520FFF730FD2CE05F2001F0CCFFF0
:1041C0005E2001F0C9FF5D2001F0C6FF5C2001F018
:1041D000C3FF542001F0C0FF562001F0BDFF552061
:1041E00001F0BAFF16E05F2001F0B6FF5E2001F09B
:1041F000B3FF5D2001F0B0FF5C2001F0ADFF542063
:10420000FFF70AFD562001F0A7FF552001F0A4FF9B
:1042100000E000BF00BF2BE5230003F016FE0A06F6
:104220001C32485E748AA0B6CCE2582001F094FF9C
:10423000512001F091FF532001F08EFF5B2001F02F
:104240008BFF5A2001F088FF592001F085FF522092
:10425000FFF7E2FCC6E05820FFF7DEFC512001F03A
:104260007BFF532001F078FF5B20FFF7D5FC5A203D
:10427000FFF7D2FC5920FFF7CFFC5220FFF7CCFC10
:10428000B0E0582001F068FF512001F065FF532095
:10429000FFF7C2FC5B2001F05FFF5A2001F05CFFDA
:1042A0005920FFF7B9FC522001F056FF9AE0582040
:1042B00001F052FF512001F04FFF532001F04CFF5D
:1042C0005B2001F049FF5A20FFF7A6FC5920FFF7B9
:1042D000A3FC522001F040FF84E05820FFF79CFC33
:1042E000512001F039FF532001F036FF5B20FFF72A
:1042F00093FC5A20FFF790FC592001F02DFF52202B
:1043000001F02AFF6EE0582001F026FF5120FFF750
:1043100083FC532001F020FF5B2001F01DFF5A2099
:10432000FFF77AFC592001F017FF522001F014FF2B
:1043300058E0582001F010FF5120FFF76DFC53208A
:1043400001F00AFF5B2001F007FF5A2001F004FF93
:10435000592001F001FF522001F0FEFE42E05820FA
:1043600001F0FAFE512001F0F7FE532001F0F4FEB7
:104370005B20FFF751FC5A20FFF74EFC5920FFF756
:104380004BFC5220FFF748FC2CE0582001F0E4FEE3
:10439000512001F0E1FE532001F0DEFE5B2001F030
:1043A000DBFE5A2001F0D8FE592001F0D5FE522044
:1043B00001F0D2FE16E0582001F0CEFE512001F0AF
:1043C000CBFE532001F0C8FE5B2001F0C5FE5A2051
:1043D000FFF722FC592001F0BFFE522001F0BCFE85
:1043E00000E000BF00BF43E4230003F02EFD0A06F7
:1043F0001C32485E748AA0B6CCE20B2001F0ACFE01
:10440000122001F0A9FE102001F0A6FE082001F004
:10441000A3FE092001F0A0FE0A2001F09DFE11205C
:10442000FFF7FAFBC6E00B20FFF7F6FB122001F0C6
:1044300093FE102001F090FE0820FFF7EDFB09200D
:10444000FFF7EAFB0A20FFF7E7FB1120FFF7E4FB89
:10445000B0E00B2001F080FE122001F07DFE102064
:10446000FFF7DAFB082001F077FE092001F074FE67
:104470000A20FFF7D1FB112001F06EFE9AE00B201D
:1044800001F06AFE122001F067FE102001F064FEC8
:10449000082001F061FE0920FFF7BEFB0A20FFF7AC
:1044A000BBFB112001F058FE84E00B20FFF7B4FBAA
:1044B000122001F051FE102001F04EFE0820FFF7FF
:1044C000ABFB0920FFF7A8FB0A2001F045FE1120F5
:1044D00001F042FE6EE00B2001F03EFE1220FFF7DD
:1044E0009BFB102001F038FE082001F035FE09206A
:1044F000FFF792FB0A2001F02FFE112001F02CFEA5
:1045000058E00B2001F028FE1220FFF785FB102059
:1045100001F022FE082001F01FFE092001F01CFE20
:104520000A2001F019FE112001F016FE42E00B20D6
:1045300001F012FE122001F00FFE102001F00CFE1F
:104540000820FFF769FB0920FFF766FB0A20FFF749
:1045500063FB1120FFF760FB2CE00B2001F0FCFD5A
:10456000122001F0F9FD102001F0F6FD082001F005
:10457000F3FD092001F0F0FD0A2001F0EDFD11200E
:1045800001F0EAFD16E00B2001F0E6FD122001F03B
:10459000E3FD102001F0E0FD082001F0DDFD092021
:1045A000FFF73AFB0A2001F0D7FD112001F0D4FDFE
:1045B00000E000BF00BF5EE4230003F046FC0A06F3
:1045C0001C32485E748AA0B6CCE23B2001F0C4FDE8
:1045D0003A2001F0C1FD392001F0BEFD382001F084
:1045E000BBFD192001F0B8FD1B2001F0B5FD1A201C
:1045F000FFF712FBC6E03B20FFF70EFB3A2001F06D
:10460000ABFD392001F0A8FD3820FFF705FB19208C
:10461000FFF702FB1B20FFF7FFFA1A20FFF7FCFA57
:10462000B0E03B2001F098FD3A2001F095FD3920E3
:10463000FFF7F2FA382001F08FFD192001F08CFD10
:104640001B20FFF7E9FA1A2001F086FD9AE03B20D3
:1046500001F082FD3A2001F07FFD392001F07CFD60
:10466000382001F079FD1920FFF7D6FA1B20FFF75B
:10467000D3FA1A2001F070FD84E03B20FFF7CCFA5A
:104680003A2001F069FD392001F066FD3820FFF77E
:10469000C3FA1920FFF7C0FA1B2001F05DFD1A20B4
:1046A00001F05AFD6EE03B2001F056FD3A20FFF785
:1046B000B3FA392001F050FD382001F04DFD1920EA
:1046C000FFF7AAFA1B2001F047FD1A2001F044FD74
:1046D00058E03B2001F040FD3A20FFF79DFA3920D9
:1046E00001F03AFD382001F037FD192001F034FDCA
:1046F0001B2001F031FD1A2001F02EFD42E03B208D
:1047000001F02AFD3A2001F027FD392001F024FDB7
:104710003820FFF781FA1920FFF77EFA1B20FFF7F8
:104720007BFA1A20FFF778FA2CE03B2001F014FD09
:104730003A2001F011FD392001F00EFD382001F082
:104740000BFD192001F008FD1B2001F005FD1A20CA
:1047500001F002FD16E03B2001F0FEFC3A2001F0E2
:10476000FBFC392001F0F8FC382001F0F5FC1920A1
:10477000FFF752FA1B2001F0EFFC1A2001F0ECFCCD
:1047800000E000BF00BF5EE4230003F05EFB0A060A
:104790001E364E667E96AEC6DEF7FB2001F0DCFCD0
:1047A000F32001F0D9FCF92001F0D6FCF82001F04B
:1047B000D3FCFF20023001F0CFFCFF20043001F0D9
:1047C000CBFCFA20FFF728FAD9E0FB20FFF724FA08
:1047D000F32001F0C1FCF92001F0BEFCF820FFF746
:1047E0001BFAFF200230FFF717FAFF200430FFF713
:1047F00013FAFA20FFF710FAC1E0FB2001F0ACFC3D
:10480000F32001F0A9FCF920FFF706FAF82001F0E7
:10481000A3FCFF20023001F09FFCFF200430FFF7D3
:10482000FBF9FA2001F098FCA9E0FB2001F094FCD0
:10483000F32001F091FCF92001F08EFCF82001F04A
:104840008BFCFF200230FFF7E7F9FF200430FFF771
:10485000E3F9FA2001F080FC91E0FB20FFF7DCF99E
:10486000F32001F079FCF92001F076FCF820FFF745
:10487000D3F9FF200230FFF7CFF9FF20043001F019
:104880006BFCFA2001F068FC79E0FB2001F064FC8D
:10489000F320FFF7C1F9F92001F05EFCF82001F0E8
:1048A0005BFCFF200230FFF7B7F9FF20043001F076
:1048B00053FCFA2001F050FC61E0FB2001F04CFCBD
:1048C000F320FFF7A9F9F92001F046FCF82001F0E8
:1048D00043FCFF20023001F03FFCFF20043001F0D8
:1048E0003BFCFA2001F038FC49E0FB2001F034FCED
:1048F000F32001F031FCF92001F02EFCF820FFF745
:104900008BF9FF200230FFF787F9FF200430FFF713
:1049100083F9FA20FFF780F931E0FB2001F01CFC5D
:10492000F32001F019FCF92001F016FCF82001F049
:1049300013FCFF20023001F00FFCFF20043001F0D7
:104940000BFCFA2001F008FC19E0FB2001F004FC4C
:10495000F32001F001FCF92001F0FEFBF82001F04A
:10496000FBFBFF200230FFF757F9FF20043001F076
:10497000F3FBFA2001F0F0FB01E0FFE700BF00BF0E
:1049800049E4230003F061FA0A061C32485E748A87
:10499000A0B6CCE2EB2001F0DFFBE22001F0DCFB73
:1049A000E12001F0D9FBE82001F0D6FBF12001F075
:1049B000D3FBEA2001F0D0FBE920FFF72DF9C6E098
:1049C000EB20FFF729F9E22001F0C6FBE12001F01E
:1049D000C3FBE820FFF720F9F120FFF71DF9EA20DB
:1049E000FFF71AF9E920FFF717F9B0E0EB2001F023
:1049F000B3FBE22001F0B0FBE120FFF70DF9E82066
:104A000001F0AAFBF12001F0A7FBEA20FFF704F96F
:104A1000E92001F0A1FB9AE0EB2001F09DFBE220F0
:104A200001F09AFBE12001F097FBE82001F094FBF4
:104A3000F120FFF7F1F8EA20FFF7EEF8E92001F0A6
:104A40008BFB84E0EB20FFF7E7F8E22001F084FB2A
:104A5000E12001F081FBE820FFF7DEF8F120FFF70D
:104A6000DBF8EA2001F078FBE92001F075FB6EE04D
:104A7000EB2001F071FBE220FFF7CEF8E12001F01E
:104A80006BFBE82001F068FBF120FFF7C5F8EA2096
:104A900001F062FBE92001F05FFB58E0EB2001F040
:104AA0005BFBE220FFF7B8F8E12001F055FBE820BE
:104AB00001F052FBF12001F04FFBEA2001F04CFB2A
:104AC000E92001F049FB42E0EB2001F045FBE22048
:104AD00001F042FBE12001F03FFBE820FFF79CF8EA
:104AE000F120FFF799F8EA20FFF796F8E920FFF7A1
:104AF00093F82CE0EB2001F02FFBE22001F02CFBDF
:104B0000E12001F029FBE82001F026FBF12001F073
:104B100023FBEA2001F020FBE92001F01DFB16E059
:104B2000EB2001F019FBE22001F016FBE12001F07F
:104B300013FBE82001F010FBF120FFF76DF8EA20ED
:104B400001F00AFBE92001F007FB00E000BF00BF15
:104B500049E4230003F079F90A061C32485E748A9E
:104B6000A0B6CCE2DB2001F0F7FAD22001F0F4FA93
:104B7000D02001F0F1FAD82001F0EEFAD92001F0AE
:104B8000EBFADA2001F0E8FAD120FFF745F8C6E0A9
:104B9000DB20FFF741F8D22001F0DEFAD02001F04F
:104BA000DBFAD820FFF738F8D920FFF735F8DA20FC
:104BB000FFF732F8D120FFF72FF8B0E0DB2001F04B
:104BC000CBFAD22001F0C8FAD020FFF725F8D82080
:104BD00001F0C2FAD92001F0BFFADA20FFF71CF881
:104BE000D12001F0B9FA9AE0DB2001F0B5FAD22029
:104BF00001F0B2FAD02001F0AFFAD82001F0ACFAFF
:104C0000D920FFF709F8DA20FFF706F8D12001F0E4
:104C1000A3FA84E0DB20FEF7FFFFD22001F09CFA2C
:104C2000D02001F099FAD820FEF7F6FFD920FEF740
:104C3000F3FFDA2001F090FAD12001F08DFA6EE056
:104C4000DB2001F089FAD220FEF7E6FFD02001F048
:104C500083FAD82001F080FAD920FEF7DDFFDA20B0
:104C600001F07AFAD12001F077FA58E0DB2001F068
:104C700073FAD220FEF7D0FFD02001F06DFAD820D1
:104C800001F06AFAD92001F067FADA2001F064FA3B
:104C9000D12001F061FA42E0DB2001F05DFAD22080
:104CA00001F05AFAD02001F057FAD820FEF7B4FFED
:104CB000D920FEF7B1FFDA20FEF7AEFFD120FEF7D4
:104CC000ABFF2CE0DB2001F047FAD22001F044FAE0
:104CD000D02001F041FAD82001F03EFAD92001F0AD
:104CE0003BFADA2001F038FAD12001F035FA16E06B
:104CF000DB2001F031FAD22001F02EFAD02001F0B1
:104D00002BFAD82001F028FAD920FEF785FFDA2007
:104D100001F022FAD12001F01FFA00E000BF00BF2D
:104D200049E4230003F091F80A061C32485E748AB5
:104D3000A0B6CCE2C32001F00FFAC22001F00CFAB9
:104D4000C12001F009FAC02001F006FAC92001F0E3
:104D500003FACB2001F000FACA20FEF75DFFC6E09F
:104D6000C320FEF759FFC22001F0F6F9C12001F07F
:104D7000F3F9C020FEF750FFC920FEF74DFFCB200E
:104D8000FEF74AFFCA20FEF747FFB0E0C32001F05C
:104D9000E3F9C22001F0E0F9C120FEF73DFFC02099
:104DA00001F0DAF9C92001F0D7F9CB20FEF734FF82
:104DB000CA2001F0D1F99AE0C32001F0CDF9C22058
:104DC00001F0CAF9C12001F0C7F9C02001F0C4F90F
:104DD000C920FEF721FFCB20FEF71EFFCA2001F0FD
:104DE000BBF984E0C320FEF717FFC22001F0B4F93D
:104DF000C12001F0B1F9C020FEF70EFFC920FEF777
:104E00000BFFCB2001F0A8F9CA2001F0A5F96EE054
:104E1000C32001F0A1F9C220FEF7FEFEC12001F07F
:104E20009BF9C02001F098F9C920FEF7F5FECB20D0
:104E300001F092F9CA2001F08FF958E0C32001F087
:104E40008BF9C220FEF7E8FEC12001F085F9C020F1
:104E500001F082F9C92001F07FF9CB2001F07CF943
:104E6000CA2001F079F942E0C32001F075F9C220AF
:104E700001F072F9C12001F06FF9C020FEF7CCFEFD
:104E8000C920FEF7C9FECB20FEF7C6FECA20FEF7FA
:104E9000C3FE2CE0C32001F05FF9C22001F05CF9F1
:104EA000C12001F059F9C02001F056F9C92001F0E4
:104EB00053F9CB2001F050F9CA2001F04DF916E06A
:104EC000C32001F049F9C22001F046F9C12001F0E8
:104ED00043F9C02001F040F9C920FEF79DFECB2028
:104EE00001F03AF9CA2001F037F900E000BF00BF35
:104EF00049E4230002F0A9FF0A061C32485E748AC6
:104F0000A0B6CCE2B32001F027F9AB2001F024F9E0
:104F1000B12001F021F9B02001F01EF9B92001F013
:104F20001BF9BB2001F018F9B220FEF775FEC6E0B0
:104F3000B320FEF771FEAB2001F00EF9B12001F0B5
:104F40000BF9B020FEF768FEB920FEF765FEBB2026
:104F5000FEF762FEB220FEF75FFEB0E0B32001F084
:104F6000FBF8AB2001F0F8F8B120FEF755FEB020B9
:104F700001F0F2F8B92001F0EFF8BB20FEF74CFE8B
:104F8000B22001F0E9F89AE0B32001F0E5F8AB2097
:104F900001F0E2F8B12001F0DFF8B02001F0DCF818
:104FA000B920FEF739FEBB20FEF736FEB22001F035
:104FB000D3F884E0B320FEF72FFEAB2001F0CCF84D
:104FC000B12001F0C9F8B020FEF726FEB920FEF7A7
:104FD00023FEBB2001F0C0F8B22001F0BDF86EE066
:104FE000B32001F0B9F8AB20FEF716FEB12001F0B6
:104FF000B3F8B02001F0B0F8B920FEF70DFEBB20E9
:1050000001F0AAF8B22001F0A7F858E0B32001F0AF
:10501000A3F8AB20FEF700FEB12001F09DF8B02010
:1050200001F09AF8B92001F097F8BB2001F094F84C
:10503000B22001F091F842E0B32001F08DF8AB20EE
:1050400001F08AF8B12001F087F8B020FEF7E4FD06
:10505000B920FEF7E1FDBB20FEF7DEFDB220FEF732
:10506000DBFD2CE0B32001F077F8AB2001F074F801
:10507000B12001F071F8B02001F06EF8B92001F014
:105080006BF8BB2001F068F8B22001F065F816E07B
:10509000B32001F061F8AB2001F05EF8B12001F01F
:1050A0005BF8B02001F058F8B920FEF7B5FDBB2041
:1050B00001F052F8B22001F04FF800E000BF00BF4D
:1050C0005EE4230002F0C1FE0A061C32485E748AC8
:1050D000A0B6CCE2A32001F03FF89A2001F03CF802
:1050E000992001F039F8A02001F036F8A92001F04C
:1050F00033F8A22001F030F8A120FEF78DFDC6E0C4
:10510000A320FEF789FD9A2001F026F8992001F0EE
:1051100023F8A020FEF780FDA920FEF77DFDA22048
:10512000FEF77AFDA120FEF777FDB0E0A32001F0A5
:1051300013F89A2001F010F89920FEF76DFDA020D9
:1051400001F00AF8A92001F007F8A220FEF764FD9B
:10515000A12001F001F89AE0A32000F0FDFF9A20C1
:1051600000F0FAFF992000F0F7FFA02000F0F4FF14
:10517000A920FEF751FDA220FEF74EFDA12000F070
:10518000EBFF84E0A320FEF747FD9A2000F0E4FF48
:10519000992000F0E1FFA020FEF73EFDA920FEF7D8
:1051A0003BFDA22000F0D8FFA12000F0D5FF6EE06B
:1051B000A32000F0D1FF9A20FEF72EFD992000F0E9
:1051C000CBFFA02000F0C8FFA920FEF725FDA220FC
:1051D00000F0C2FFA12000F0BFFF58E0A32000F0C4
:1051E000BBFF9A20FEF718FD992000F0B5FFA02024
:1051F00000F0B2FFA92000F0AFFFA22000F0ACFF4A
:10520000A12000F0A9FF42E0A32000F0A5FF9A2012
:1052100000F0A2FF992000F09FFFA020FEF7FCFC09
:10522000A920FEF7F9FCA220FEF7F6FCA120FEF76C
:10523000F3FC2CE0A32000F08FFF9A2000F08CFFFD
:10524000992000F089FFA02000F086FFA92000F03F
:1052500083FFA22000F080FFA12000F07DFF16E078
:10526000A32000F079FF9A2000F076FF992000F04B
:1052700073FFA02000F070FFA920FEF7CDFCA22054
:1052800000F06AFFA12000F067FF00E000BF00BF50
:105290005EE4230002F0D9FD0A061C32485E748ADF
:1052A000A0B6CCE2932000F057FF8A2000F054FF14
:1052B000882000F051FF902000F04EFF912000F078
:1052C0004BFF922000F048FF8920FEF7A5FCC6E0C6
:1052D0009320FEF7A1FC8A2000F03EFF882000F01A
:1052E0003BFF9020FEF798FC9120FEF795FC922062
:1052F000FEF792FC8920FEF78FFCB0E0932000F0CF
:105300002BFF8A2000F028FF8820FEF785FC9020E4
:1053100000F022FF912000F01FFF9220FEF77CFC9E
:10532000892000F019FF9AE0932000F015FF8A20F1
:1053300000F012FF882000F00FFF902000F00CFF1B
:105340009120FEF769FC9220FEF766FC892000F0B0
:1053500003FF84E09320FEF75FFC8A2000F0FCFE50
:10536000882000F0F9FE9020FEF756FC9120FEF711
:1053700053FC922000F0F0FE892000F0EDFE6EE07C
:10538000932000F0E9FE8A20FEF746FC882000F01A
:10539000E3FE902000F0E0FE9120FEF73DFC92201D
:1053A00000F0DAFE892000F0D7FE58E0932000F0EC
:1053B000D3FE8A20FEF730FC882000F0CDFE90203E
:1053C00000F0CAFE912000F0C7FE922000F0C4FE5B
:1053D000892000F0C1FE42E0932000F0BDFE8A204B
:1053E00000F0BAFE882000F0B7FE9020FEF714FC13
:1053F0009120FEF711FC9220FEF70EFC8920FEF7AB
:105400000BFC2CE0932000F0A7FE8A2000F0A4FE05
:10541000882000F0A1FE902000F09EFE912000F078
:105420009BFE922000F098FE892000F095FE16E089
:10543000932000F091FE8A2000F08EFE882000F07C
:105440008BFE902000F088FE9120FEF7E5FB922075
:1054500000F082FE892000F07FFE00E000BF00BF68
:105460005EE4230002F0F1FC0A061F38516A839CB7
:10547000B5CEE7FDFC2000F06FFEFD2000F06CFED5
:10548000FE2000F069FEFF2000F066FEFF200830DD
:1054900000F062FEFF20063000F05EFEFF200730C5
:1054A000FEF7BAFBE3E0FC20FEF7B6FBFD2000F0C0
:1054B00053FEFE2000F050FEFF20FEF7ADFBFF2064
:1054C0000830FEF7A9FBFF200630FEF7A5FBFF2002
:1054D0000730FEF7A1FBCAE0FC2000F03DFEFD20F6
:1054E00000F03AFEFE20FEF797FBFF2000F034FEAE
:1054F000FF20083000F030FEFF200630FEF78CFB66
:10550000FF20073000F028FEB1E0FC2000F024FE70
:10551000FD2000F021FEFE2000F01EFEFF2000F026
:105520001BFEFF200830FEF777FBFF200630FEF75A
:1055300073FBFF20073000F00FFE98E0FC20FEF721
:105540006BFBFD2000F008FEFE2000F005FEFF20B2
:10555000FEF762FBFF200830FEF75EFBFF200630FF
:1055600000F0FAFDFF20073000F0F6FD7FE0FC20A0
:1055700000F0F2FDFD20FEF74FFBFE2000F0ECFDF9
:10558000FF2000F0E9FDFF200830FEF745FBFF207B
:10559000063000F0E1FDFF20073000F0DDFD66E0A1
:1055A000FC2000F0D9FDFD20FEF736FBFE2000F0C8
:1055B000D3FDFF2000F0D0FDFF20083000F0CCFD2F
:1055C000FF20063000F0C8FDFF20073000F0C4FDCA
:1055D0004DE0FC2000F0C0FDFD2000F0BDFDFE20F0
:1055E00000F0BAFDFF20FEF717FBFF200830FEF7A2
:1055F00013FBFF200630FEF70FFBFF200730FEF7FE
:105600000BFB34E0FC2000F0A7FDFD2000F0A4FD22
:10561000FE2000F0A1FDFF2000F09EFDFF200830DD
:1056200000F09AFDFF20063000F096FDFF200730C5
:1056300000F092FD1BE0FC2000F08EFDFD2000F04C
:105640008BFDFE2000F088FDFF2000F085FDFF208F
:105650000830FEF7E1FAFF20063000F07DFDFF2064
:1056600000E003E0073000F077FD00E000BF00BF7E
:105670003EE4230002F0E9FB0A061C32485E748A0D
:10568000A0B6CCE2EC2000F067FDE42000F064FD61
:10569000EE2000F061FDEF2000F05EFDF62000F04E
:1056A0005BFDF42000F058FDED20FEF7B5FAC6E0F2
:1056B000EC20FEF7B1FAE42000F04EFDEE2000F001
:1056C0004BFDEF20FEF7A8FAF620FEF7A5FAF4202E
:1056D000FEF7A2FAED20FEF79FFAB0E0EC2000F012
:1056E0003BFDE42000F038FDEE20FEF795FAEF20B8
:1056F00000F032FDF62000F02FFDF420FEF78CFACA
:10570000ED2000F029FD9AE0EC2000F025FDE420DA
:1057100000F022FDEE2000F01FFDEF2000F01CFD48
:10572000F620FEF779FAF420FEF776FAED2000F085
:1057300013FD84E0EC20FEF76FFAE42000F00CFD8E
:10574000EE2000F009FDEF20FEF766FAF620FEF7E6
:1057500063FAF42000F000FDED2000F0FDFC6EE0A7
:10576000EC2000F0F9FCE420FEF756FAEE2000F001
:10577000F3FCEF2000F0F0FCF620FEF74DFAF420E9
:1057800000F0EAFCED2000F0E7FC58E0EC2000F02F
:10579000E3FCE420FEF740FAEE2000F0DDFCEF2011
:1057A00000F0DAFCF62000F0D7FCF42000F0D4FC86
:1057B000ED2000F0D1FC42E0EC2000F0CDFCE42034
:1057C00000F0CAFCEE2000F0C7FCEF20FEF724FA40
:1057D000F620FEF721FAF420FEF71EFAED20FEF780
:1057E0001BFA2CE0EC2000F0B7FCE42000F0B4FC45
:1057F000EE2000F0B1FCEF2000F0AEFCF62000F04F
:10580000ABFCF42000F0A8FCED2000F0A5FC16E0B5
:10581000EC2000F0A1FCE42000F09EFCEE2000F063
:105820009BFCEF2000F098FCF620FEF7F5F9F42041
:1058300000F092FCED2000F08FFC00E000BF00BF04
:105840003EE4230002F001FB0A061C32485E748A23
:10585000A0B6CCE2DC2000F07FFCD52000F07CFC80
:10586000D62000F079FCDF2000F076FCE62000F086
:1058700073FCDD2000F070FCDE20FEF7CDF9C6E001
:10588000DC20FEF7C9F9D52000F066FCD62000F038
:1058900063FCDF20FEF7C0F9E620FEF7BDF9DD204E
:1058A000FEF7BAF9DE20FEF7B7F9B0E0DC2000F031
:1058B00053FCD52000F050FCD620FEF7ADF9DF20D8
:1058C00000F04AFCE62000F047FCDD20FEF7A4F9DA
:1058D000DE2000F041FC9AE0DC2000F03DFCD52009
:1058E00000F03AFCD62000F037FCDF2000F034FC5A
:1058F000E620FEF791F9DD20FEF78EF9DE2000F0BC
:105900002BFC84E0DC20FEF787F9D52000F024FC96
:10591000D62000F021FCDF20FEF77EF9E620FEF71E
:105920007BF9DD2000F018FCDE2000F015FC6EE0B5
:10593000DC2000F011FCD520FEF76EF9D62000F037
:105940000BFCDF2000F008FCE620FEF765F9DD2007
:1059500000F002FCDE2000F0FFFB58E0DC2000F04D
:10596000FBFBD520FEF758F9D62000F0F5FBDF2031
:1059700000F0F2FBE62000F0EFFBDD2000F0ECFB96
:10598000DE2000F0E9FB42E0DC2000F0E5FBD52062
:1059900000F0E2FBD62000F0DFFBDF20FEF73CF951
:1059A000E620FEF739F9DD20FEF736F9DE20FEF7B6
:1059B00033F92CE0DC2000F0CFFBD52000F0CCFB4D
:1059C000D62000F0C9FBDF2000F0C6FBE62000F087
:1059D000C3FBDD2000F0C0FBDE2000F0BDFB16E0C5
:1059E000DC2000F0B9FBD52000F0B6FBD62000F09B
:1059F000B3FBDF2000F0B0FBE620FEF70DF9DD2061
:105A000000F0AAFBDE2000F0A7FB00E000BF00BF13
:105A10009FE3230002F019FA0A061C32485E748ADA
:105A2000A0B6CCE2CC2000F097FBC52000F094FBA0
:105A3000C72000F091FBCF2000F08EFBCE2000F0BD
:105A40008BFBCD2000F088FBC620FEF7E5F8C6E012
:105A5000CC20FEF7E1F8C52000F07EFBC72000F067
:105A60007BFBCF20FEF7D8F8CE20FEF7D5F8CD206F
:105A7000FEF7D2F8C620FEF7CFF8B0E0CC2000F059
:105A80006BFBC52000F068FBC720FEF7C5F8CF20F0
:105A900000F062FBCE2000F05FFBCD20FEF7BCF8EB
:105AA000C62000F059FB9AE0CC2000F055FBC52041
:105AB00000F052FBC72000F04FFBCF2000F04CFB62
:105AC000CE20FEF7A9F8CD20FEF7A6F8C62000F0FC
:105AD00043FB84E0CC20FEF79FF8C52000F03CFBA0
:105AE000C72000F039FBCF20FEF796F8CE20FEF756
:105AF00093F8CD2000F030FBC62000F02DFB6EE0C7
:105B0000CC2000F029FBC520FEF786F8C72000F066
:105B100023FBCF2000F020FBCE20FEF77DF8CD2028
:105B200000F01AFBC62000F017FB58E0CC2000F074
:105B300013FBC520FEF770F8C72000F00DFBCF2047
:105B400000F00AFBCE2000F007FBCD2000F004FBA4
:105B5000C62000F001FB42E0CC2000F0FDFAC52099
:105B600000F0FAFAC72000F0F7FACF20FEF754F859
:105B7000CE20FEF751F8CD20FEF74EF8C620FEF7F6
:105B80004BF82CE0CC2000F0E7FAC52000F0E4FA56
:105B9000C72000F0E1FACF2000F0DEFACE2000F0BE
:105BA000DBFACD2000F0D8FAC62000F0D5FA16E0D6
:105BB000CC2000F0D1FAC52000F0CEFAC72000F0CA
:105BC000CBFACF2000F0C8FACE20FEF725F8CD2082
:105BD00000F0C2FAC62000F0BFFA00E000BF00BF2C
:105BE000B7E2230002F031F90A061C32485E748ADB
:105BF000A0B6CCE2B42000F0AFFAB52000F0ACFAC9
:105C0000B62000F0A9FAB72000F0A6FABE2000F0F6
:105C1000A3FABC2000F0A0FABD20FDF7FDFFC6E00E
:105C2000B420FDF7F9FFB52000F096FAB62000F099
:105C300093FAB720FDF7F0FFBE20FDF7EDFFBC2083
:105C4000FDF7EAFFBD20FDF7E7FFB0E0B42000F06C
:105C500083FAB52000F080FAB620FDF7DDFFB7200B
:105C600000F07AFABE2000F077FABC20FDF7D4FFEE
:105C7000BD2000F071FA9AE0B42000F06DFAB52072
:105C800000F06AFAB62000F067FAB72000F064FA74
:105C9000BE20FDF7C1FFBC20FDF7BEFFBD2000F018
:105CA0005BFA84E0B420FDF7B7FFB52000F054FAAA
:105CB000B62000F051FAB720FDF7AEFFBE20FDF789
:105CC000ABFFBC2000F048FABD2000F045FA6EE0C2
:105CD000B42000F041FAB520FDF79EFFB62000F099
:105CE0003BFAB72000F038FABE20FDF795FFBC2044
:105CF00000F032FABD2000F02FFA58E0B42000F096
:105D00002BFAB520FDF788FFB62000F025FAB72062
:105D100000F022FABE2000F01FFABC2000F01CFAAE
:105D2000BD2000F019FA42E0B42000F015FAB520C9
:105D300000F012FAB62000F00FFAB720FDF76CFF62
:105D4000BE20FDF769FFBC20FDF766FFBD20FDF713
:105D500063FF2CE0B42000F0FFF9B52000F0FCF95F
:105D6000B62000F0F9F9B72000F0F6F9BE2000F0F7
:105D7000F3F9BC2000F0F0F9BD2000F0EDF916E0D9
:105D8000B42000F0E9F9B52000F0E6F9B62000F003
:105D9000E3F9B72000F0E0F9BE20FDF73DFFBC209D
:105DA00000F0DAF9BD2000F0D7F900E000BF00BF35
:105DB000CFE1230002F049F80A061C32485E748ADB
:105DC000A0B6CCE2A42000F0C7F99C2000F0C4F9F2
:105DD000A62000F0C1F9A72000F0BEF9AE2000F027
:105DE000BBF9AC2000F0B8F9A520FDF715FFC6E01F
:105DF000A420FDF711FF9C2000F0AEF9A62000F0D2
:105E0000ABF9A720FDF708FFAE20FDF705FFAC209A
:105E1000FDF702FFA520FDF7FFFEB0E0A42000F093
:105E20009BF99C2000F098F9A620FDF7F5FEA7202D
:105E300000F092F9AE2000F08FF9AC20FDF7ECFEF7
:105E4000A52000F089F99AE0A42000F085F99C20B3
:105E500000F082F9A62000F07FF9A72000F07CF97D
:105E6000AE20FDF7D9FEAC20FDF7D6FEA52000F050
:105E700073F984E0A420FDF7CFFE9C2000F06CF9BC
:105E8000A62000F069F9A720FDF7C6FEAE20FDF7B9
:105E9000C3FEAC2000F060F9A52000F05DF96EE0D3
:105EA000A42000F059F99C20FDF7B6FEA62000F0D2
:105EB00053F9A72000F050F9AE20FDF7ADFEAC205D
:105EC00000F04AF9A52000F047F958E0A42000F0BE
:105ED00043F99C20FDF7A0FEA62000F03DF9A72085
:105EE00000F03AF9AE2000F037F9AC2000F034F9B8
:105EF000A52000F031F942E0A42000F02DF99C200B
:105F000000F02AF9A62000F027F9A720FDF784FE6B
:105F1000AE20FDF781FEAC20FDF77EFEA520FDF74B
:105F20007BFE2CE0A42000F017F99C2000F014F96F
:105F3000A62000F011F9A72000F00EF9AE2000F025
:105F40000BF9AC2000F008F9A52000F005F916E0E7
:105F5000A42000F001F99C2000F0FEF8A62000F03B
:105F6000FBF8A72000F0F8F8AE20FDF755FEAC20B6
:105F700000F0F2F8A52000F0EFF800E000BF00BF4D
:105F8000E7E0230001F061FF0A061C32485E748AD4
:105F9000A0B6CCE2942000F0DFF88D2000F0DCF811
:105FA0008F2000F0D9F8972000F0D6F89E2000F05E
:105FB000D3F8952000F0D0F89620FDF72DFEC6E02E
:105FC0009420FDF729FE8D2000F0C6F88F2000F008
:105FD000C3F89720FDF720FE9E20FDF71DFE9520BB
:105FE000FDF71AFE9620FDF717FEB0E0942000F0B2
:105FF000B3F88D2000F0B0F88F20FDF70DFE97204C
:1060000000F0AAF89E2000F0A7F89520FDF704FE06
:10601000962000F0A1F89AE0942000F09DF88D20E1
:1060200000F09AF88F2000F097F8972000F094F88D
:106030009E20FDF7F1FD9520FDF7EEFD962000F086
:106040008BF884E09420FDF7E7FD8D2000F084F8C4
:106050008F2000F081F89720FDF7DEFD9E20FDF7F0
:10606000DBFD952000F078F8962000F075F86EE0E2
:10607000942000F071F88D20FDF7CEFD8F2000F008
:106080006BF8972000F068F89E20FDF7C5FD95207D
:1060900000F062F8962000F05FF858E0942000F0DD
:1060A0005BF88D20FDF7B8FD8F2000F055F89720A4
:1060B00000F052F89E2000F04FF8952000F04CF8C8
:1060C000962000F049F842E0942000F045F88D2039
:1060D00000F042F88F2000F03FF89720FDF79CFD7C
:1060E0009E20FDF799FD9520FDF796FD9620FDF782
:1060F00093FD2CE0942000F02FF88D2000F02CF878
:106100008F2000F029F8972000F026F89E2000F05C
:1061100023F8952000F020F8962000F01DF816E0F6
:10612000942000F019F88D2000F016F88F2000F070
:1061300013F8972000F010F89E20FDF76DFD9520D4
:1061400000F00AF8962000F007F800E000BF00BF5A
:1061500000BF00BF70BD000030B50146C3175B0F24
:106160005B18DB10094CE35C0246C417640FA418EB
:10617000E410E400051B0124AC402343C417640F62
:106180006418E410014D2B5530BD0000C8220020DA
:1061900010B5044630222146002000F0F2F810BD70
:1061A00010B500F0C1FF08210C48FCF71CF90120D4
:1061B00002F094FE04210948FCF717F9042002F0CC
:1061C0008DFE04210548FCF70EF9042002F086FE3E
:1061D00008210248FCF709F910BD0000C00C00407E
:1061E00010B500F0A1FF08210A48FCF7FEF80120D5
:1061F00002F074FE04210748FCF7F7F8042002F0CF
:106200006DFE04210348FCF7EEF8042002F066FE60
:1062100010BD0000C00C004070B5002508211348D7
:10622000FCF7E3F800F070FF80241BE004210F4826
:10623000FCF7DBF8012002F051FE08210B48FCF7C7
:10624000C8F8012803D128462043054602E0284625
:10625000A043054604210548FCF7C5F8042002F0D8
:106260003DFE6410002CE1D1284670BDC00C0040FA
:1062700070B5044600F058FF00251EE08020204045
:10628000002804D008211548FCF7AFF803E00821E6
:106290001248FCF7A8F86006040E0A2002F01EFE61
:1062A00004210E48FCF7A1F80A2002F017FE042191
:1062B0000A48FCF798F8681CC5B2082DDEDB0A20F6
:1062C00002F00CFE04210548FCF78FF80A2002F0CA
:1062D00005FE04210148FCF786F870BDC00C0040A3
:1062E00010B500F021FF08210A48FCF77EF80421D0
:1062F0000848FCF77AF8052002F0F0FD082105486F
:10630000FCF771F8042002F0E9FD04210148FCF7D4
:106310006AF810BDC00C004010B500F005FF082160
:106320000A48FCF760F8042002F0D8FD0421074871
:10633000FCF75BF8042002F0D1FD08210348FCF7CC
:1063400054F8052002F0CAFD10BD0000C00C00404A
:10635000F8B507460D4616460024FFF7C1FF7C201E
:10636000FFF786FF3846FFF783FF00BF04E0285D94
:10637000FFF77EFF601CC4B2B442F8DBFFF7CCFF2E
:10638000F8BDF8B507460D4616460024FFF7A8FFEE
:106390007C20FFF76DFF8020FFF76AFF3846FFF78C
:1063A00067FF00BF04E0285DFFF762FF601CC4B216
:1063B000B442F8DBFFF7B0FFF8BD08B5022002F0E9
:1063C00065FD032168460170012269468220FFF7BE
:1063D000BFFF032168460170022002F057FD012231
:1063E00069468420FFF7B4FF08BD000004488069B7
:1063F000C007C00F002801D0012070470020FCE733
:106400000034014010B500F00BF8012807D1FFF768
:10641000EDFF012803D100F00FF802F051FB10BD91
:106420000448406940210840002801D001207047FD
:106430000020FCE7003401404020014948617047DA
:106440000034014000200C490978002903D00A4992
:106450000978092901D101210843084989784907A8
:10646000490F042907D0054989784907490F0329AD
:1064700001D0022108437047140000201C010020B5
:10648000F0B589B00021C848C1720173002600250B
:106490000CE0C648405D412807D1C448691C405CF7
:1064A000412802D1C148461964256D1C642DF0DBDA
:1064B000002E38D00027002507E0705DBC49485504
:1064C0000846405DC019C7B26D1C192DF5DB707E02
:1064D000B84228D1B07E162825D1B078012816D12F
:1064E000F078012802DDF078B249C871002504E097
:1064F000301D415DB04841556D1C142DF8DB307ED8
:10650000002805D0317EAB482030817100E000BF0B
:106510000120A8494870032088707821A5482330BD
:10652000017100214171A5A1A048F9F765FE064659
:10653000002E7DD0A2A13046F9F75EFE0446002C65
:10654000F7D00025641C04E06D1C641C0A2D00DDDE
:1065500002E060786828F7D100BF782195482330A1
:10656000017100214171E07A0690207B617B090274
:10657000401880B20790607DA17D0902401880B26A
:106580000890E07E05900027002504E0601C405D37
:10659000C019C7B26D1C07980D308542F6DB07980D
:1065A0002018807BB84243D160786828FBD1A07A5C
:1065B0006828F8D1FCF754F9824880797E491C3963
:1065C00048738048C07888737E480079C8737D48D6
:1065D000007808747B48407848747A4880788874DA
:1065E000069805284ED17849089888424AD18021DA
:1065F00005980840002803D1207F002814D013E01C
:10660000002505E020461C30405D694948556D1C59
:10661000102DF7DB664A6D491046FAF709FC64480D
:106620000078002800D000BF63491C39C87D00E015
:10663000B8E0897D000208435F4A1C3A517E127E11
:1066400009021143884203DA00215A48203041727E
:1066500059491C39C87D897D00020843401C80B21D
:1066600055491C398875000AC875594800780428AE
:1066700005DB57480078001F5549087002E00020EC
:1066800053490870069801288DD1524908988842CC
:1066900089D14C484078A17C884210DCA17C4948D3
:1066A0004078C01C81421ADD464840786030A17CA9
:1066B000401A092813DD0120474908700FE04148BE
:1066C0004178A07CC01C814209DDA07C60303D493E
:1066D0004978401A092802DD01203F4908703E48E8
:1066E0000078012825D1A07B3C490870E07B4870E8
:1066F000207C8870607CC870A07C0871E07C487148
:10670000084640790979354AD27800920191029081
:10671000324882784078049030480078012149035B
:10672000401801230390049900F03AFE00202A4902
:1067300008702BA0FBF764FFFF20F53002F0A6FBEA
:10674000FF20F53002F0A2FBFF20F53002F09EFBA7
:10675000FF20F53002F09AFBFF2101312248F9F7C2
:1067600040FDFF2101311148F9F73BFD00210E48A2
:10677000C17201730F482030417200201449087023
:1067800001210D481C3881750021C1750020174971
:106790000870174908701749087000211548203003
:1067A0008174C17409B0F0BD671D0020671C002012
:1067B0002F1E0020781D0020BF1D00202B5200003E
:1067C0002C0000001A06002060840000381700200A
:1067D0000F06002050A400003506002022060020ED
:1067E0004154434C4F534500671B002002060020D4
:1067F00004060020611A002070B504460025FCF74D
:1068000097FB1048007C002819D000210D48017426
:10681000FF210131401AF9F7E4FC0A48C27A0A491B
:10682000FF380138F9F7C4FC122C02D1FFF728FE1B
:1068300004E000210348C172017300BF00BF284675
:1068400070BD0000671D0020671B0020F8B5002404
:1068500088E0A000454909680F5CA0004349096829
:10686000085CA100414A1268891849784840A10093
:106870003E4A1268891889784840A1003B4A12684C
:106880008918C97805464D40A00038490968085C58
:10689000A100364A126889184978484006463046B1
:1068A00003F004FC0646A00030490968085C314644
:1068B00069404840A1002D4A12685054A0002B495D
:1068C000096840184078A100284A12688918897818
:1068D00048400646304603F0E9FB0646A00023493F
:1068E000096840184078314669404840A1001F4A75
:1068F000126889184870A0001C49096840188078FF
:10690000A1001A4A12688918C978484006463046DC
:1069100003F0CCFB0646A0001449096840188078B3
:10692000314669404840A100104A126889188870B1
:10693000A0000E4909684018C078784006463046E5
:1069400003F0B4FB0646A000084909684018C07867
:10695000314669404840A100044A12688918C8704D
:10696000601CC4B2042C00DA73E7F8BD34040020C4
:1069700010B5002000F002F9012820D1002000F01D
:1069800009F900BF0E4840780007C00F002812D157
:106990000B49497B082291430831094A5173090781
:1069A000C90FC9000822114008460549497891439A
:1069B0000143034A517000BF02A001F00BFA10BD61
:1069C0001C010020BFAAB8C7B1A8BEAF0D0A0000C5
:1069D000002805DBC206D20E01219140014A116058
:1069E0007047000080E100E0002805DBC206D20EFF
:1069F00001219140014A11607047000000E100E070
:106A000010B5002819DB1A4A03231B02D218830889
:106A10009B00D2588307DC0EFF23A3409A438B07C9
:106A20001B0E8407E40EA3401A43114B03242402D7
:106A30001B198408A4001A5118E00E4A03071B0F03
:106A4000083B9B089B00D2588307DC0EFF23A34022
:106A50009A438B071B0E8407E40EA3401A43054B91
:106A60000407240F083CA408A4001A5110BD00001C
:106A700000E100E01CED00E07FB506460D4614463F
:106A80006A4629463046FBF7D9FB0098A84217D141
:106A90006846C079002813D1002C03D1684640799C
:106AA00000280DD1012C03D168464079012807D177
:106AB00068468079002803D168460079012813D000
:106AC000029500206946C873002C01D1487302E08A
:106AD00001206946487300216846817301210173D2
:106AE00002A93046FBF73CFC7FBD00000146064A88
:106AF0001068931502469A4310461A460A401043FE
:106B0000014A106070470000002000400146054A1D
:106B10001068800880008A07920F1043014A1060B5
:106B200070470000002000400146064A10685315D7
:106B300002469A4310461A460A401043014A106022
:106B4000704700000020004010B504466068FFF761
:106B5000EBFF207AFFF7CAFF0121490260688842F3
:106B600002D1206900F01CF80349E0680861206840
:106B7000FFF7CCFF10BD000000ED00E00146044827
:106B800080680840002801D0012070470020FCE701
:106B9000002000400149886070470000002000404C
:106BA0000146054A5068800880008A07920F10430A
:106BB000014A5060704700000020004010B502F00C
:106BC0008BFF03F013F803F07BF803F025F900F0D6
:106BD00005F802F0A9FF02F0BBFF10BD10B50821B7
:106BE0003048FBF7F6FB00281CD104212D48FBF7A9
:106BF000FAFB002414E0FF2101312A48C038FBF7DA
:106C0000F2FBC82002F042F9FF2101312548C038CB
:106C1000FBF7EBFBC82002F039F9FCF713FA641C10
:106C2000032CE8DB02211F48C038FBF7D2FB012808
:106C300037D1002414E0FF2101311A48C038FBF796
:106C4000D2FBC82002F022F9FF2101311548C038DB
:106C5000FBF7CBFBC82002F019F9FCF7F3F9641C31
:106C6000052CE8DB80210F48FBF7B3FB012818D186
:106C7000002414E0FF2101310A48C038FBF7B3FBC0
:106C8000C82002F003F9FF2101310648C038FBF7A4
:106C9000ACFBC82002F0FAF8FCF7D4F9641C062C0F
:106CA000E8DB10BD800D0040F8B507460D461646DE
:106CB000FFF716FB6420FFF7DBFA3846FFF7D8FA38
:106CC000FFF70EFB6520FFF7D3FA002406E0FFF77D
:106CD000A3FA2855FFF764FA601CC4B2701EA042E4
:106CE000F5DCFFF799FA2855FFF77AFAFFF714FB5E
:106CF000F8BDF8B507460D461646FFF7F1FA6420D1
:106D0000FFF7B6FA3846FFF7B3FA002404E0285D2F
:106D1000FFF7AEFA601CC4B2B442F8DBFFF7FCFA2E
:106D2000F8BD00000146064A5068062302469A4311
:106D3000104606220A401043014A50607047000086
:106D400000280040012806D1064949680122114364
:106D5000044A516005E00349496849084900014A6D
:106D600051607047002800400146064A106806231B
:106D700002469A43104606220A401043014A106018
:106D80007047000000280040012806D10649096824
:106D900001221143044A116005E0034909684908CA
:106DA0004900014A1160704700280040C104C90C25
:106DB000014A1163704700000010014002488069D9
:106DC0008006800E704700000010014002484069B4
:106DD0008006800E704700000010014002480069E4
:106DE0004006400E70470000001001400248006A53
:106DF000C006C00E70470000001001400248C06885
:106E00004006400E70470000001001400248C06973
:106E10004007400F70470000001001400148406AE1
:106E2000C0B270470010014010B501210648FAF7C2
:106E3000E7FC002204210548FFF71EFE002208217E
:106E40000248FFF719FE10BD07000001C00C00400A
:106E500010B50B48407A012805D1FFF7F3FA032853
:106E600001D100F039FA00F011F8012807D100F043
:106E700019F80120034908700348FBF7BFFC10BD57
:106E8000E40300203C040020050000200448806842
:106E900008210840002801D0012070470020FCE7AD
:106EA000001001400820014988607047001001402F
:106EB00000B50146FFF7A2FF4871FFF78FFF087189
:106EC000FFF784FFC870FFF779FF8870FFF78EFF28
:106ED0004870FFF7A3FF0870FFF798FF887100BDA7
:106EE00010B50D488078012815D10CA000F072FF74
:106EF000002406E00D48015D0DA000F06BFF601C52
:106F000084B205480088A042F4DC0BA000F062FFC8
:106F100000200149887010BD441600204D43553CA7
:106F20002D6D6F6462757320000000004412002014
:106F300030782530327820000D0A000070B5002628
:106F40000920FAF781FF05461A488078A84216D032
:106F5000022001F09BFF0CE00920FAF775FF0546BF
:106F6000022001F093FF3046711C8EB2642800DDD0
:106F700004E00920FAF768FFA842EDD100BF0E48EF
:106F8000281A84B2002C13D00A4804800520FAF78E
:106F90009DFF00210520FAF731FF07490520FAF788
:106FA0005BFF01210520FAF729FF012001498870C4
:106FB00070BD0000441600204412002001460869FC
:106FC000C007C00F002801D0012070470020FCE757
:106FD0000146086902221040002801D001207047B4
:106FE0000020FCE701468869704741617047000056
:106FF00010B500F065F8012828D102202449086165
:1070000000F06AF800BF234800798007C00F00280D
:1070100012D12049097C02229143891C1D4A117416
:107020008907C90F49000222114008461949097908
:1070300091430143174A117100BF0120164908709E
:107040000020C87315A000F0C5FE1FE000F04AF84C
:1070500001281BD10E49086100F050F800BF0D480F
:1070600000798007C00F00280CD00A48007902215F
:1070700088430849087111200B49088011210B48E9
:10708000F9F73CFF00BF0AA000F0A4FE10BD00000D
:10709000002801401C010020FA000020EFAEB5E7F7
:1070A000C7B7D1B90D0A0000F8000020280400205D
:1070B000EFAEB5E7C7B7D1B9BBD6B8B40D0A00007B
:1070C0000448C06802210840002801D00120704710
:1070D0000020FCE70028014002200149C8607047F9
:1070E000002801400448C068C007C00F002801D034
:1070F000012070470020FCE70028014001200149E1
:10710000C86070470028014010B501210448FAF713
:1071100077FB002208210348FCF727F810BD000088
:1071200007000001C00C004010B501210448FAF727
:1071300067FB002208210348FFF79EFC10BD0000FA
:1071400007000001C00C004010B500BF1E4800F051
:107150005EFD0028FAD067211B4800F0B3FD00BF98
:10716000194800F054FD0028FAD018480078801C17
:10717000C1B2154800F0A6FD00BF134800F047FD5E
:107180000028FAD011480088801C0004010E0E4827
:1071900000F098FD00240BE000BF0B4800F037FD25
:1071A0000028FAD00A48015D074800F08BFD641CF6
:1071B00006480088801C8442EEDB00BF024800F0D5
:1071C00026FD0028FAD010BD007001400006002006
:1071D0002F1E002024490968487823490968497905
:1071E000214A12685170204909684A7A1E49096883
:1071F0004A711D4909684A7B1B4909684A721A4944
:107200000968487318490968887817490968897AAC
:10721000154A126891701449096888721249096800
:107220008879114909688A7B0F4909688A710E4972
:10723000096888730C490968C8780B490968C97BD3
:10724000094A1268D17008490968CA7A064909686A
:10725000CA7305490968CA7903490968CA720249AB
:107260000968C871704700003404002010B5044656
:1072700021460A48FFF7B9FE00BF0848FFF7A8FEFD
:107280000028FAD000BF0548FFF798FE0028FAD082
:107290000248FFF7A7FE0446E0B210BD004C0140D3
:1072A00070B5002413E000250DE0A900094A12681A
:1072B0008918085D01F004FFA900064A12688918C0
:1072C0000855681CC5B2042DEFDB601CC4B2042C49
:1072D000E9DB70BD340400201FB500240120FAF75B
:1072E00097FB07200002FAF7A5FB032001F0CEFD73
:1072F0000120FAF7D3F905E019200002844200D3F7
:1073000004E0641CFAF7DEF90028F5D000BF012084
:1073100000900020019002900120694608736846A1
:10732000FAF766FB014801F08DFD1FBD001BB70099
:107330000148006870470000B0030020014802497E
:107340000860704700127A003806002010B572B647
:10735000FBF780FE104801F075FD0A2001F096FD54
:10736000FBF7F8FE0120FFF70FFD0620FFF7DAFC20
:107370000020FFF7E7FCFAF708FC01210748FAF7BD
:107380003FFA0020FFF712FD00210448FAF738FA0F
:10739000FBF758FE62B610BD00127A000200000131
:1073A000FFB583B006460C4615460C9F01204749A1
:1073B0000870FFF739FDF6B2F0210E980840001171
:1073C0000A2148430E990907090F40183C2803DA9F
:1073D00069460E98087102E0002069460871F021A4
:1073E0000D98084000110A2148430D990907090F1B
:1073F00040183C2803DA69460D98487102E00020E5
:1074000069464871F020384000110A214843390785
:10741000090F4018182802DA6846877102E0002038
:107420006946887169460698C871F02028400011A5
:107430000A2148432907090F401820280CDAF020B8
:10744000284000110A2148432907090F4018002845
:1074500002DD6846057202E0012069460872F020EC
:10746000204000110A2148432107090F40180D2828
:107470000CDAF020204000110A2148432107090FAF
:107480004018002802DD6846447202E00120694687
:107490004872F020304000110A2148433107090F9B
:1074A0004018642802DA69468E7202E015206946A7
:1074B0008872072201A90020FFF71BFC0A2001F0B7
:1074C000E5FC00200149087007B0F0BD3606002039
:1074D00070B504460D4601218806FAF791F903209C
:1074E000FAF780F90120FAF76BF90120F9F754FF58
:1074F0000020F9F775FF601EF9F7B6FF681EF9F76F
:1075000045FF1B20FFF764FA01211B20FFF778FAE3
:107510001B20FFF769FA0120F9F772FF0120F9F744
:107520004DFFF9F79BFF70BD10B50D4800F012FB41
:10753000012813D10A4800F057FB01280ED103207F
:10754000FAF7C4FC00210320FAF758FC0549032090
:10755000FAF782FC01210320FAF750FC10BD00006D
:1075600000680140671B002010B50D4800F0F2FADA
:10757000012813D10A4800F037FB01280ED105205D
:10758000FAF7A4FC00210520FAF738FC054905208C
:10759000FAF762FC01210520FAF730FC10BD00006B
:1075A00000780140F8220020F3B585B00F46059819
:1075B000F9F7DFF805463846F9F7DBF806462946BD
:1075C000F8F7FBFE04907F21C9050498F9F7E2F96A
:1075D00013D20498F9F786F905460022094BF8F70B
:1075E000CFFF0022084B01910090F8F725FF03918F
:1075F0000290F9F739F9044600E00024204607B06C
:10760000F0BD00000000F03F0000E03F30B505464F
:107610000C462846616800F02BFA2846A16800F065
:1076200036FA2846E16800F026FA2846616900F03B
:107630005FFA617C284600F0A5FA217C284600F01C
:10764000AEFA2178284600F090FA6178284600F0DA
:10765000B3FAA178284600F0BBFAA17E284600F0D4
:107660002EFAE17E284600F069FAA17C284600F057
:107670001AFA217E284600F048FA617E284600F07A
:1076800050FA30BD00B597B001216D48FAF7B8F84F
:107690000022FF2101316B48F9F756FD002201213C
:1076A00049026848F9F750FD002201218902654826
:1076B000FFF7E2F9012189026248FAF796FEE1201C
:1076C00040021490012110A80175002141758175B7
:1076D0000DA8F9F753FF0DAA14A95B4800F0C0F8F4
:1076E0000E20FFF775F90121574800F0DCF9012160
:1076F000554800F00AFA544800F081FA0121534835
:10770000FAF77EF80120FAF7AFFB05216846017110
:107710000120400303908010049003204002059054
:10772000002006904A4802904A480990002007909D
:10773000002108A8417081700121C1701520FFF758
:1077400047F90520FAF7C2FB01A8FAF7C7FB0121A8
:107750003E48FAF755F80120FAF786FB0121384830
:10776000FAF74EF80022012136484030F9F7ECFCD8
:107770000022022133484030F9F7E6FC00220121C3
:1077800089033048FFF778F900220121C9032D4809
:10779000FFF772F9002016904B20C00114900121D0
:1077A00010A801750021417581750DA8F9F7E6FE55
:1077B0000DAA14A9284800F053F80A20FFF708F989
:1077C000FF21254800F076FA234800F01CFA012139
:1077D000214800F0E4F90A20FFF706F901211E48CC
:1077E00000F079F901211C4800F05DF901211A48E7
:1077F00000F08BF9184800F002FA0921684601717F
:107800000120400303908010049040100590002058
:1078100006900F480290114809900020079000211F
:1078200008A8417081700121C1701520FFF7D0F8C0
:107830000920FAF74BFB01A8FAF750FB17B000BD7F
:1078400007000001000C0040007801400400000225
:10785000FF03000048060020006801404412002099
:1078600070B588B006460C4615467A48864228D13F
:10787000A068F9F773FF0120F9F75CFF0121764852
:10788000F9F7BEFFA068002804D0012808D002281C
:1078900015D10EE0A9682068FFF786FE02900FE080
:1078A0000120FAF723F8E9682068FFF77DFE0290CF
:1078B00006E029682068FFF777FE029000E000BF2D
:1078C00063E06648864229D1A068F9F769FF012084
:1078D000F9F752FF01216048401CF9F791FFA068B9
:1078E000002804D0042808D0082815D10EE0A96883
:1078F0002068FFF759FE02900FE00120F9F7F6FF2C
:10790000E9682068FFF750FE029006E029682068C9
:10791000FFF74AFE029000E000BF36E05048864282
:107920000AD101214C48801CF9F76AFFA968206838
:10793000FFF73AFE029028E04A4886420AD1012128
:107940004548C01CF9F75CFFA9682068FFF72CFECA
:1079500002901AE0444886420AD101213E48001DA7
:10796000F9F74EFFA9682068FFF71EFE02900CE0B1
:107970003E48864209D101213748401DF9F740FFB2
:10798000A9682068FFF710FE02902079012810D125
:10799000402003906079012802D1102004903FE03C
:1079A0006079022802D12020049039E00020049060
:1079B00036E02079022810D18020039060790128D8
:1079C00002D1102004902BE06079022802D12020FF
:1079D000049025E00020049022E0207900280FD1B7
:1079E00003906079012802D11020049018E060799A
:1079F000022802D12020049012E0002004900FE021
:107A0000C02003906079012802D11020049007E083
:107A10006079022802D12020049001E00020049027
:107A2000A079002801D1069002E0FF2001300690E5
:107A3000002168460171417181714175017581773D
:107A4000C17781750177417701A93046FFF7DEFDE7
:107A500008B070BD0020014008000003006801402C
:107A6000006C01400070014000740140007801404A
:107A70008AB28261704710B50A46016830240B460D
:107A8000A3431946302313401943016010BD10B5BC
:107A90000A460168C0240B46A3431946C02313407D
:107AA0001943016010BD012904D1026802231A4361
:107AB000026003E0026802239A43026070470129D2
:107AC00004D1026808231A43026003E00268082315
:107AD0009A4302607047012904D102680B041A43DB
:107AE000026004E0026801231B049A4302607047AD
:107AF00010B50A460168FF2401340B46A34319461A
:107B0000234613401943016010BD012904D10268C6
:107B100001231A43026003E0026852085200026027
:107B20007047012904D102684B041A43026004E043
:107B3000026801235B049A4302607047012904D163
:107B4000026804231A43026003E0026804239A4394
:107B50000260704701464868FF2201321040002849
:107B600001D0012070470020FCE7012904D14268C0
:107B70000B021A43426004E04268FF2301339A4338
:107B800042607047012904D142688B021A43426067
:107B900004E0426801239B029A4342607047012936
:107BA00004D14268CB021A43426004E042680123D8
:107BB000DB029A4342607047012904D142680223E4
:107BC0001A43426003E0426802239A4342607047CE
:107BD000012904D1426801231A43426003E042684C
:107BE000520852004260704701468868FF22013205
:107BF0001040002801D0012070470020FCE7FF2141
:107C00000131816070470121C902816070470146DE
:107C10008868C007C00F002801D0012070470020ED
:107C2000FCE70000F8B504460D46164600270BE0B9
:107C3000E95D204600F046F800BF2046FFF7E7FF69
:107C40000028FAD0781C87B2B742F1DB0E48844294
:107C500001D10EA005E00E48844201D10DA000E044
:107C60000CA001460DA000F0B5F8002705E0E95D85
:107C70000DA000F0AFF8781C87B2B742F7DB0CA07C
:107C800000F0A8F8F8BD0000007801405043000063
:107C90000068014055415254310000004D43552DBC
:107CA0003E25732000000000307825303278200017
:107CB0000D0A00000A46C168090A0902D3B2194335
:107CC000C1607047CA05D20D4261704710B50F48B8
:107CD0008078012818D10EA000F07CF8002406E07E
:107CE0000E48015D0EA000F075F8601C84B20749D3
:107CF0004878097800020843A042F1DC0AA000F0AD
:107D000069F800200149887010BD0000480A002071
:107D10004D43553C2D5043200000000048060020F4
:107D200030782530327820000D0A0000012806D175
:107D30000649496A01221143044A516205E0034998
:107D4000496A49084900014A5162704700F80140F8
:107D50000146064A506A0E2302469A4310460E22F6
:107D60000A401043014A50627047000000F8014089
:107D700000B507484368180CD94389B2884203D13B
:107D8000D8B200F019F802E01F2000F015F800BD8D
:107D900040FBFF1F012806D1064949698022114393
:107DA000044A516105E00349496980229143014A2F
:107DB0005161704700F801400146054A5069800949
:107DC00080018A06920E1043014A506170470000FC
:107DD00000F801400FB410B503A9044B044A0298FF
:107DE00000F00AF910BC08BC04B018473D90000030
:107DF0003C0600200FB410B504A9074B02AA039853
:107E000000F0FAF8044602A9002000F091FC204698
:107E100010BC08BC04B01847318700002021020CB8
:107E200001D010211046020A01D01046083902097B
:107E300001D01046091F820801D01046891E420851
:107E400001D0881E7047081A704730B47446641E0B
:107E50002578641CAB4204D3635D5B00E31830BC3F
:107E600018471D46F8E702E008C8121F08C1002A9B
:107E7000FAD170477047002001E001C1121F002AAB
:107E8000FBD17047F0B51FB486B00998089A030D6E
:107E90000021024314D05148514A18185043051488
:107EA0001198012810981AD0281A401C00264D4F0E
:107EB0004D49009601910490002812DA444211E0E5
:107EC0001198012449A3012801D11098C1430698B3
:107ED000119A84600360C26041600BB0F0BD404203
:107EE000E4E70446210500203F4A001C514103916C
:107EF000029012E0E00707D032463B460199009815
:107F0000F8F74CFB0191009032463B46104619466B
:107F1000F8F744FB06460F466410002CEAD104989B
:107F2000039B0028029A0999089806DAF8F736FBAD
:107F3000019B009AF8F732FB05E0F8F797FB019BED
:107F4000009AF8F793FB04460E460022284BF8F7F8
:107F5000F1FC03D80020C043014607E00022254B76
:107F600020463146F8F768FAF8F79CFC102409E03F
:107F7000002C0ADB0A220023F8F7EAF8079B3032CC
:107F80001A55641E02460A43F2D11122641C079B53
:107F9000121B1C19119B012B03D0012308430ED186
:107FA0000AE0084304D0112010900020119077E7D8
:107FB0001098151A6D1E0BE01098824202DD002306
:107FC0006D1C03E0824201DA00236D1E002BEED00F
:107FD000069811998260C16030C07EE701FCFFFF06
:107FE000104D0000000014400000F03F3000000081
:107FF0000000F0430000E03FFFB597B006460025C3
:1080000018E2252877D100242746FD49049400E092
:108010000443761C32780120203A90400842F7D180
:1080200030782A280ED002223078014630390929CA
:1080300016D804990A235943303940181443761C42
:108040000490F1E7189802C804911890002904DA06
:108050000120400304434842049002200443761C5C
:1080600030782E2814D1042004437078761C2A28F6
:1080700009D11898761C80C8189009E00A214F434E
:10808000303FC719761C3078014630390929F5D9B7
:1080900030786C2810D006DC4C281AD068280ED016
:1080A0006A2817D104E0742813D07A2812D110E07E
:1080B0000120400504430CE00121090501E00321F2
:1080C00009050C437178814203D101200005241871
:1080D000761C761C3078119066280BD013DC58285B
:1080E0007DD009DC00287BD04528F6D04628F4D086
:1080F00047281AD1A5E118E0632835D0642870D04C
:10810000652812D19DE170286CD008DC6728F1D079
:1081100069287BD06E280DD06F2806D1BAE073286D
:108120002ED0752871D0782859D01A9A199990476D
:108130006D1C7EE16002400F022809D003280DD09B
:108140000428189801680DD00D60001D189070E18A
:108150001898EA1701680D604A60F6E718980168F8
:108160000D80F2E70D70F0E718986A4601781172F9
:10817000001D18900020507202A80090012005E018
:10818000189802C8189000200091C04361070DD5CF
:10819000002101E00199491C0191B94212DA8142A2
:1081A000F8DB009A515C0029F4D10BE0002101E0DA
:1081B0000199491C01918142FADB019A0099895C7D
:1081C0000029F5D1019904981A9B471A214638468F
:1081D000199A00F097FA0199401945180BE04FE001
:1081E0002CE113E04EE0009800990078491C0091C2
:1081F0001A9A199990470198401E0190401CF2D19B
:10820000214638461A9B199A10E137E00A200021CE
:10821000009001916002410F022907D0189A01CA0B
:108220001892C2179446032908D00AE01898C01D76
:10823000C108C90005C91891944607E000B2C217E9
:108240009446042902D140B2C1178C4600226146EF
:10825000944506DA0A460021404291418C462D2180
:1082600002E0210504D52B216A461173012103E0A8
:10827000E10701D02021F7E7029155E00A200AE04A
:10828000102008E0102000900021042004430191F8
:10829000082703E008200021019100906002410FAF
:1082A000022907D0189A01CA18920022944603297D
:1082B00008D008E01898C01DC108C90005C9189168
:1082C000944603E080B2042900D1C0B2002102919B
:1082D000210729D51199702906D0009A1021019BF8
:1082E0004A401A4305D00EE040216A46117301212D
:1082F00008E06146014306D030216A4611731199A6
:10830000517302210291009A0821019B4A401A43AD
:108310000AD16146014301D1610705D530216A4682
:10832000117301217F1E02911199582904D035A1A2
:108330000E910DA90D910DE037A1F9E76146019B62
:10834000009AF7F705FF0E9B8C469B5C0D9A521E18
:108350000D92137061460143F0D10D9805A9081ADA
:1083600020300190600703D501200004844300E021
:1083700001270198874201DD381A00E000200199A9
:1083800000904118029809180498401A0490E003DC
:1083900006D421461A9B199A049800F0B3F945199E
:1083A000002706E003A81A9AC05D199990476D1C32
:1083B0007F1C02988742F5DBE0030CD521461A9B0F
:1083C000199A049800F09EF9451904E01A9A302091
:1083D000199990476D1C0099481E00900029F5DC02
:1083E00008E00D980D990078491C0D911A9A199979
:1083F00090476D1C0199481E01900029F1DC63E152
:10840000092801003031323334353637383961626A
:10841000636465660000000030313233343536372E
:1084200038394142434445460000000000F05AF903
:108430004519761C3078002800D0E2E528461BB0AC
:10844000F0BD600700D406271898C01DC108C900F8
:1084500048680A680831C30FDB071891190001D07A
:108460009CA108E0210501D59BA104E0E10701D012
:108470009AA100E09AA1430011985B081091652829
:108480000CD006DC452809D046281DD0472841D10C
:1084900041E0662818D067283CD13CE00021112F2C
:1084A00001DB112000E0781C0191009008A911A8BF
:1084B000FFF7E8FC139905910021119A15927F1C92
:1084C00012980197009150E00120C007039001200D
:1084D000019008A9009711A8FFF7D4FC139A1499EA
:1084E00005920022119B009212981593059A019211
:1084F000002901D0104602E0791C40180190381A7A
:1085000001D5019804E04042401E0090781C019083
:10851000C01B029043E0012F00DA01270021112F38
:1085200001DD112000E038460191009008A911A852
:10853000FFF7A8FC13990591119A00211298159242
:108540000091019721070CD40599B94201DB0199EB
:1085500000E00191012904DD159A491E515C302982
:1085600006D0B84201DA011D05DA0121029115E0B9
:108570000199491EEDE7002805DC0099411800919A
:108580000199091A03E0019A411C914200DD019111
:108590000099401A401C02900120C0070390200758
:1085A00006D402990198814202DB0020C043029068
:1085B00000206946C87707AF012103980337C90730
:1085C000884224D0022011902B201290039800287A
:1085D0000CDA404203902D20129007E00A21039804
:1085E000F7F78CFD30317F1E039039701199481ECA
:1085F00011900029F2DC03980028EFD1791E12981F
:1086000008703078202108404530BF1E387006A819
:10861000C01BC01D039010980078002800D00120D6
:10862000019941180298C01709180398091804986D
:10863000401A401E0490E00306D421461A9B199A62
:10864000049800F05FF8451910980078002803D0CE
:108650001A9A199990476D1CE00324D521461A9B5C
:10866000199A049800F04EF845191CE0009800286B
:1086700007DB00990598884203DD1598405C19993D
:1086800001E0199930201A9A904700986D1C401CFF
:1086900000900298401E0290002804D11A9A2E20C1
:1086A000199990476D1C0199481E01900029DDDC45
:1086B00005E038781A9A7F1C199990476D1C039928
:1086C000481E03900029F4DC21461A9B199A04984D
:1086D000ACE600002D0000002B0000002000000090
:1086E00000000000F8B5044600251E461746880421
:1086F00004D405E039462020B0476D1C641EF9D52E
:108700002846F8BDFFB50446002581B01E46C803C3
:1087100001D5302700E02027880404D505E038463D
:108720000399B0476D1C641EF9D5284605B0F0BD0D
:108730000A68531C0B60107070470000F0B585B0DC
:108740000446002004902248808AA0421ED220497C
:10875000898A601AF8F70DF800901E4801680098A1
:10876000F7F72BFE01901C4801680198F7F78FFD81
:108770000746F8F7B7F805460022184BF7F700FF51
:1087800003910290F8F7EAF804901DE01049898AF5
:10879000081BF7F7EEFF00900E4801680098F7F706
:1087A0000CFE01900C4801680198F7F7C5FD0746DB
:1087B000F8F798F805460022084BF7F7E1FE039119
:1087C0000290F8F7CBF80490049805B0F0BD0000D3
:1087D00040FBFF1F0C000020100000200000E03FC5
:1087E000F0B587B00446002713490A20085EF7F762
:1087F000C7FF05460022114BF7F738FF039102909F
:108800000D49098961430846F7F7CEFF0546002266
:108810000B4BF7F72BFF01910090039B029AF7F7A0
:108820000BFE05910490F7F7FBFF0746002F00DAD7
:108830000027384607B0F0BD80FAFF1F00005940FE
:1088400000408F4010B5002400BFF8F7A7FA0128B8
:1088500001D1002010BD2046641C401C0028F4D12A
:108860000120F7E770B50446606880470546E07868
:108870004007400F002802DD2088401C2080E0785F
:10888000C009A8421CD0E07838218843E1788906E5
:10889000490F491CC900382211400843E070800686
:1088A000400F032810DBE07880218843E901802213
:1088B00011400843E070E07838218843E07003E01D
:1088C000E07838218843E070E0784007400F0300EB
:1088D000FFF7BBFA06042856A7F4D1F4E078C009E4
:1088E000E1784906C90F884216D1A078F021884363
:1088F000A070A068002802D02046A1688847002008
:108900002080A07800090001401CA070E078C00819
:10891000C000401CE07004E0A078F0218843803063
:10892000A070CBE0E078C009E1784906C90F884221
:1089300012D0A078F02188431030A070E0680028A1
:1089400002D02046E168884700202080E078C008F7
:10895000C000801CE07012E0208864280FDDA07841
:10896000F02188435030A070E069002802D02046F2
:10897000E1698847E078C008C000401DE0709DE0D4
:10898000E078C009E1784906C90F884220D1A07873
:10899000F0218843A070A068002802D02046A1687A
:1089A0008847A07800090001A178491C0907090F30
:1089B0000843A0702069002802D02046216988471A
:1089C00000202080E078C008C000C01CE07027E0D4
:1089D00020880F2824DDA0780007000F01280BD184
:1089E000A078F02188433030A0706069002813D04F
:1089F0002046616988470FE0A0780007000F022831
:108A00000AD1A078F02188434030A070A0690028E6
:108A100002D02046A1698847E078C008C000E07015
:108A20004CE0E078C009E1784906C90F88421AD0C5
:108A3000A078F02188431030A070E068002802D0B0
:108A40002046E168884720880F2807DA0020208028
:108A5000E078C008C000801CE0700BE0E078C0083F
:108A6000C000E07006E020880F2803DDE078C00831
:108A7000C000E07022E0E078C009E1784906C90F43
:108A800088420BD1A078F02188436030A070206A22
:108A9000002812D02046216A88470EE0A078F021F5
:108AA00088431030A070E068002802D02046E168BA
:108AB0008847E078C008C000E07000BF00BF70BD0C
:108AC00010B50548046803E02046FFF7CBFE646A52
:108AD000002CF9D110BD0000AC050020F7B584B022
:108AE000074616463B480068039000253A48006850
:108AF00002900020019039480078002822D03848A0
:108B0000007800281ED13748826928466D1C8000F5
:108B10003A5034484069441E33480068844211D3B7
:108B200031480068314909684018A0420AD3102D25
:108B300008D20598854205D228466D1C80003C501D
:108B4000012001902648007800280CD00398864226
:108B500001D2039E07E0029903984018B04202D266
:108B60000299039846182DE03068041FE007C00FF3
:108B7000002800D125E03068441E1B480068001D15
:108B800084421DD318480068184909684018A0425B
:108B900016D3102D14D2201F00F0C8F900280FD0D2
:108BA000059885420CD2022D06D10198002803D0E9
:108BB0007868A04200D104E028466D1C80003C503B
:108BC00000BF361D029903984018B042CCD8284601
:108BD00007B0F0BDB0050020B4050020C10500209D
:108BE000C205002078190020B8050020BC0500202F
:108BF000F0B58FB00E4635462C4620224D4907A8C9
:108C0000F7F7D6FA4C4807684C48006806904C487D
:108C10000078002809D14B4A4BA14DA0FFF7DAF8A4
:108C200053A0FFF7D7F800BFFEE7524800780028AE
:108C300009D0444A50A146A0FFF7CCF84CA0FFF75A
:108C4000C9F800BFFEE701204A4908704DA0FFF7B0
:108C5000C1F847A0FFF7BEF800F0D2F84A49C86A49
:108C6000FFF7B8F842A0FFF7B5F82035BD4203D3AF
:108C700006983818A84202D20120444908702A46B2
:108C80003846069900F070F94048007800284BD12A
:108C90003D49086BFFF79EF835A0FFF79BF83C496C
:108CA0002068086060684860A0688860E068C86004
:108CB0002069086160694861A0698861E069C861EC
:108CC0000846C068324A0A999268099B0193029249
:108CD000039104902E48406800902D48089B02683C
:108CE0002CA00799FFF776F821A0FFF773F8284822
:108CF000C069274A0E9992690D9B019302920391D4
:108D0000049023484069009021480C9B026921A0EF
:108D10000B99FFF75FF816A0FFF75CF828A0FFF7A4
:108D200059F813A0FFF756F8284600F089FE0FB057
:108D3000F0BD000080A40000B0050020B4050020B4
:108D4000C00500206CA40000696E69745F6F6B0041
:108D500028257329206861732061737365727420FC
:108D60006661696C65642061742025732E000000C3
:108D70000D0A0000C1050020216F6E5F6661756CF1
:108D80007400000000000000C0A30000C205002025
:108D900078190020202025733A20253038782020AB
:108DA00025733A2025303878202025733A20253045
:108DB0003878202025733A202530387800000000CC
:108DC0003D3D3D3D3D3D3D3D3D3D3D3D3D3D3D3DD3
:108DD0003D3D3D3D3D3D3D3D3D3D3D3D3D3D3D3DC3
:108DE0003D3D3D3D3D3D3D3D3D3D3D3D3D3D3D3DB3
:108DF0003D3D3D3D3D3D3D3D3D3D3D3D3D3D00001D
:108E000010B50549054B064A48680649FEF7E2FFDA
:108E100005A0FEF7DFFF10BDC0A30000C8180020AA
:108E2000A8180020881800200D0A000000B501468F
:108E3000FEF77EFA024600BFFEF77AFA5318984210
:108E4000FAD300BD10B504460C480068C021884321
:108E50000A49086008460068C021084307490860BD
:108E600007492046F7F74AF906490870084600788E
:108E70007D21C90048430449088010BD00240040FA
:108E800040420F0000000020020000200146114A6D
:108E900012884A43104B5A6100229A611A4612699D
:108EA00001231A430C4B1A6100BF0B4A1069C20719
:108EB000D20F002A04D0012212040240002AF4D06A
:108EC000054A126952085200034B1A6100229A6146
:108ED000704700000200002000E000E00146114A57
:108EE00012784A43104B5A6100229A611A4612695D
:108EF00001231A430C4B1A6100BF0B4A1069C207C9
:108F0000D20F002A04D0012212040240002AF4D019
:108F1000054A126952085200034B1A6100229A61F5
:108F2000704700000000002000E000E010B501469E
:108F30000B884A881F20C00210401F24E402A04270
:108F400006D118400F242403A04201D1012010BDF6
:108F5000FF200002104047242402A04201D101203A
:108F6000F5E70020F3E7000070B505460E4614460D
:108F70001D48007800281CD01C480078002808D024
:108F80001B4988692146FEF725FF1AA0FEF722FF3C
:108F900007E01749C8692146FEF71CFF15A0FEF738
:108FA00019FFAC4201D22C4603E0A819A04200D21E
:108FB000AC190F490869FEF70DFF0EA0FEF70AFF76
:108FC00008E021460CA02268FEF704FF09A0FEF786
:108FD00001FF241DA819A042F3D80EA0FEF7FAFE47
:108FE00004A0FEF7F7FE70BDC2050020C3050020F7
:108FF000C0A300000D0A00002020616464723A20C2
:109000002530387820202020646174613A20253092
:10901000387800003D3D3D3D3D3D3D3D3D3D3D3DC4
:109020003D3D3D3D3D3D3D3D3D3D3D3D3D3D3D3D70
:109030003D3D3D3D3D3D3D3D0000000070B50446D9
:109040000D46E1B20548FEF73DFE00BF0348FEF7BE
:10905000DEFD0028FAD0204670BD000000780140F7
:1090600010B5002823D0124B0022001F196803E01E
:10907000814203D80A4649680029F9D1002A0AD05A
:109080001368841A9C4204D10068181810601046B6
:1090900002E0506000E01860002907D002680B1A57
:1090A000934203D10B68D21802604968416010BD39
:1090B0004006002001460148405C7047BEA1000008
:1090C00001460148405C7047BEA00000F0B591B079
:1090D000FE48407C012808D1FD4909688900FD4A05
:1090E0008818F9F75BF80F9001E000200F90F7481F
:1090F000007C012809D1F649096889007D22D20047
:109100008818F9F730F80E9001E000200E90EF4833
:10911000007D012808D1EE4909688900EE4A8818C7
:10912000F9F707F80B9001E000200B90E748407D2D
:10913000012812D1E64909688900E84A8818F8F739
:10914000F8FF0A90E1492039886AF7F712FB079087
:109150000A99F7F7F5F80A9001E000200A90DB4839
:10916000C07C012808D1DA4909688900DC4A8818DE
:10917000F8F7DFFF0D9001E000200D90D348807CD0
:10918000012808D1D24909688900D64A8818F8F719
:10919000D0FF0C9001E000200C90CD490968C90077
:1091A000D14A8818F8F76CFF04460D46C84909688B
:1091B000C900CE4A8818F8F763FF06460F46C4492F
:1091C0000968C900CA4A8818F8F75AFF0991089037
:1091D000BF490968C74A8818F8F722FFC6490870CE
:1091E000BB490968C54A8818F8F71AFFC249487090
:1091F000B7490968C24A8818F8F712FFBE49887053
:10920000B3490968BF4A8818F8F70AFFBA49C87015
:10921000AF490968BC4A8818F8F702FFB6490871D7
:10922000AB490968B94A8818F8F7FAFEB24948719B
:1092300020462946F7F718FB0190F7F7B5FA2246C2
:109240002B4603910290F7F7A1F90022B04B05914C
:109250000490F7F7A3F907910690F7F705FB81B2A1
:10926000A5488171090AC17120462946F7F7FCFA21
:10927000A14908310790F6F7F2FF00221346204675
:109280002946F7F743FB2FD222462B460020014602
:10929000F7F776F904460D4620462946F7F7E4FA33
:1092A0000190F7F781FA22462B4603910290F7F7D7
:1092B0006DF90022964B05910490F7F76FF907912D
:1092C0000690F7F7D1FA81B28B488171090AC17112
:1092D00020462946F7F7C8FA0121C90708438649FD
:1092E00008310790F6F7BBFF30463946F7F7BCFA6E
:1092F0000190F7F759FA32463B4603910290F7F78F
:1093000045F90022824B05910490F7F747F9079140
:109310000690F7F7A9FA81B277480173090A4173F9
:1093200030463946F7F7A0FA73490E310790F6F741
:1093300096FF09990898F7F797FA0190F7F734FA2A
:1093400003910290099B089AF7F720F90022704BCD
:1093500005910490F7F722F907910690F7F784FA40
:1093600081B265488174090AC17409990898F7F7B0
:109370007BFA614914310790F6F771FF00215E48CE
:109380000176417601461A310F98F6F768FF002101
:1093900059488177C177014620310E98F6F75FFF73
:1093A0000D98F7F728FA0490F7F7E3F905900D996F
:1093B000F6F7C2FF57490690F6F7C2FF0790F7F796
:1093C0001AFA81B24C4820300171090A41710D9896
:1093D000F7F711FA484926310790F6F740FF0C9845
:1093E000F7F709FA0490F7F7C4F905900C99F6F726
:1093F000A3FF48490690F6F7A3FF0790F7F7FBF99C
:1094000081B23D4822300172090A41720C98F7F787
:10941000F2F939492C310790F6F721FF36493031FE
:109420000B98F6F71CFF344934310A98F6F717FF0A
:10943000394A1378194653781B02194393781B0451
:109440001943D278120611430846F7F7BBF9049086
:10945000F7F784F9304A05901378184653781B02C1
:10946000184393781B041843D27812061043014620
:109470000598F6F761FF29490690F6F761FF079016
:10948000F7F7A0F9C1B21C4820300176224A1378C0
:10949000194653781B02194393781B041943D27859
:1094A000120611430846F7F78DF9C1B21248203071
:1094B0004176194A121D1378194653781B02194335
:1094C00093781B041943D278120629E0B0220020B9
:1094D000DC0500206810000068290000E81C00007E
:1094E00068420000E835000088A90000A87A000062
:1094F00018920000685B0000DD1D0020885E0000FF
:10950000A8610000C8640000E8670000086B000064
:109510000088C34000401C46C31900200000C84218
:1095200011430846F7F74EF90490F7F717F9414A47
:1095300005901378184653781B02184393781B0440
:109540001843D2781206104301460598F6F7F4FE48
:1095500039490690F6F7F4FE0790F7F733F9C1B2F0
:1095600036488176334A1378194653781B021943DB
:1095700093781B041943D278120611430846F7F773
:1095800021F9C1B22D48C1762A4A121D1378194615
:1095900053781B02194393781B041943D27812069F
:1095A00011430846F7F70EF90490F7F7D7F8214A68
:1095B000121D05901378184653781B0218439378B0
:1095C0001B041843D2781206104301460598F6F79B
:1095D000B3FE19490690F6F7B3FE0790F7F7F2F8D5
:1095E000C1B216480177134A121D137819465378F1
:1095F0001B02194393781B041943D27812061143B6
:109600000846F7F7DFF8C1B20C48417702461E3230
:1096100000200146F6F72CFE084A263200200146BB
:10962000F6F726FE0021054822300173417311B080
:10963000F0BD0000C71900200000C842FD1D002039
:10964000002204E003780B70401C491C521C502A75
:10965000F8DB7047F8B505463A22BA49BA4800F037
:1096600089F9002D7ED1B848807E802108400028ED
:1096700043D1002418E0FFF729FD20465022504333
:109680003A30B04A8118B148FFF7DAFFB0480068B5
:10969000401CAF49086008460068AE49884202D3C2
:1096A0000020AB490860641C042CE4DBFF207B3005
:1096B000A94908800021A348A74A128881540024A0
:1096C0000BE0A048A4490988405C9E49095D401808
:1096D0009C49A14A12888854641C9F48008884428F
:1096E000EFDB1621974A9C480088401C1154FDF777
:1096F0002BFD01219948417222E1002418E0FFF777
:10970000E5FC2046502250433A308E4A81188F485B
:10971000FFF796FF8E480068401C8D490860084698
:1097200000688C49884202D3002089490860641C83
:10973000042CE4DB80218A4881760F27152600243B
:109740000AE021011B317F4BCA1821011B31C818C7
:109750008449F7F783FB641C701C8442F1DBFF2013
:109760008B3000E025E0C01B7B4908800021754854
:10977000794A1288815400240BE07248764909889E
:10978000405C7049095D40186E49734A12888854DC
:10979000641C714800888442EFDB1621694A6E48D8
:1097A0000088401C1154FDF7CFFC01216B48417229
:1097B000C6E06548807E80210840002849D1002409
:1097C00018E0FFF783FC2046502250433A305D4AB0
:1097D00081185E48FFF734FF5D480068401C5C4913
:1097E0000860084600685B49884202D30020584957
:1097F0000860641C5C4800788442E2DB5A480078C8
:10980000502148433A305449088000204D49524A7B
:109810001288885400240CE04A484F490988405C6B
:109820004849095D4018C1B246484B4A12888154E4
:10983000641C494800888442EEDB1621414A4648B0
:109840000088401C1154FDF77FFC01214348417200
:1098500076E0002418E0FFF739FC20465022504300
:109860003A30384A81183948FFF7EAFE384800682C
:10987000401C37490860084600683649884202D3D0
:10988000002033490860641C374800788442E2DBDA
:10989000802135480078502250433A30294A1154EB
:1098A000002409E0002130480078502250433B302A
:1098B0000019244A1154641C2C4800780F21081AFE
:1098C000A042EFDC00240AE021011B311D4BCA1825
:1098D00021011B31C8182349F7F7C0FA641C24483A
:1098E0000078401C8442EFDB1F4800785021484339
:1098F0004A301E490978401A17490880002011494A
:10990000154A1288885400240BE00E481249098831
:10991000405C0C49095D40180A490F4A1288885476
:10992000641C0D4800888442EFDB1621054A0A4872
:109930000088401C1154FDF707FC012107484172C3
:10994000F8BD00002F1E0020A31D0020DD1D0020FB
:10995000DC050020EE02000000060020981D00201B
:109960008F1F002038170020ED0500203004002054
:109970003104002010B5002304E004780C70401C72
:10998000491C5B1C9342F8DB10BD000010B5044677
:1099900021460548FEF796F900BF0348FEF737F960
:1099A0000028FAD010BD000000680140FDF7CEFC91
:1099B000F7F7D0FAFDF766FEF7F766FAF9F75AFB04
:1099C000F7F76EFC00F0BCFA00F0B2FA01E0FDF728
:1099D000F5F8FCE7F0B50B30C108C900144F0026BC
:1099E000144A0FE003688B420BD38B4205D95C1AF3
:1099F0004318456830C3083B00E04368136002C069
:109A000004E0021D10680028ECD13046002803D184
:109A10003868002801D00020F0BD064A06481060D2
:109A2000064A121AD208D20044C001203860D7E793
:109A300044060020400600200C24002008340020AA
:109A400070B592B006460025402102A8F6F7C9FB82
:109A50003246102102A8FFF741F80546002410E025
:109A6000A10002AB5A58E1006118134BC81813A1AA
:109A7000FEF7C0F92021E000201808300E4A1154EA
:109A8000641CAC42ECD3002D0DD00B48E9006B18E0
:109A90000C4900900CA2086A0D49FEF79BF90DA035
:109AA000FEF798F906E00749486AFEF793F909A01E
:109AB000FEF790F912B070BDE81800202530386C20
:109AC00078000000C0A300002E617866000000004E
:109AD000881800200D0A000010B5FDF729FC09497F
:109AE0000968401A084988420BD9FDF721FC05494D
:109AF0000860FF2101310548F8F779FC04A0FEF762
:109B000069F910BDB4030020581B0000C00C0040D0
:109B100063697263756C6174652074756E206F6E15
:109B2000206C65640D0A000010B5FDF701FC0649C4
:109B30000968401A0549884205D9FDF7F9FB024931
:109B40000860F8F78DFE10BDBC0300201027000050
:109B500010B5F9F731FAFDF7F1F9FEF7B7F8FDF7AF
:109B6000BFF9FDF7E5FB1A490968401A194988420F
:109B70002CD9FDF7DDFB1649086001218902164842
:109B8000F8F733FC012215491548FEF74BF801217F
:109B9000C90211484030F8F728FC012149030E485A
:109BA0004030F8F722FC7D20C000FFF73FF901218B
:109BB00089030948F8F719FC08220A490A48FEF700
:109BC00031F8012189030448F8F70DFC10BD0000AD
:109BD000C0030020581B0000000C0040D8030020E8
:109BE00000780140D90300200068014010B5202111
:109BF0002548F8F7EEFB002805D10821224840301F
:109C0000F8F7F3FB04E008211F484030F8F7EBFBBE
:109C1000012189031C48F8F7DCFB002806D001214C
:109C2000C9031948F8F7D5FB00282CD13220FFF7DB
:109C30002DF9012189031448F8F7CBFB00280ED138
:109C400012A0FEF7C7F880210F484038F8F7CDFB87
:109C500040210D484038F8F7C8FBF8F7DFFB012139
:109C6000C9030948F8F7B5FB00280CD101210648C3
:109C7000F8F7B9FBF8F72CFB0120400200F0DCF903
:109C80000BA0FEF7A7F810BD400D00405475726E92
:109C90005F4F6E20706F77657220332E33762061B0
:109CA0006E642073656E6420677072730D0A000025
:109CB0006C6F776572206D6F64656C200D0A000013
:109CC00010B500F0E5F93A490860084600683949DE
:109CD0000968884206D00520FFF7D8F800F0D8F9C7
:109CE0003349086032480068002808D031480068CD
:109CF000002804D1FDF71CFB2F49086052E02C48D6
:109D0000006800284ED12B48006800284AD0FDF793
:109D10000FFB29490968401A28490860084600686D
:109D20002749884217D201212648F8F752FB01281B
:109D30000DD1C1022448F8F758FB0121C90322487C
:109D4000F8F753FB012149031F48F8F74EFB1FA00A
:109D5000FEF740F826E0194800687D218901884215
:109D600008D2164800684910884203D91DA0FEF7A2
:109D700031F817E0114800687D218901884211D32C
:109D80001EA0FEF727F80121C9020F48F8F72DFBA6
:109D9000012189030C48F8F728FB012149030A48EF
:109DA000F8F723FB024800680249086010BD000074
:109DB000CC030020D0030020C4030020C8030020EF
:109DC000C409000000FC0140400C004053686F7261
:109DD0007420707265737320646574656374656460
:109DE0002E0A00006C6F6E672070726573732064BA
:109DF000657465637465642E0A0000004C6F6E67BD
:109E0000206C6F6E67207072657373206465746573
:109E1000637465642E0A000070B5FDF789FA28495D
:109E20000968401A2749884249D9FDF781FA24492F
:109E30000860F8F72BFC04462349F6F710FAF8F708
:109E400075FC04462049091FF6F709FAF8F7BEFC2D
:109E50001E4908601C48F6F7EAF90646F6F742FD87
:109E6000044622460B461AA0FDF7B4FF1648001F11
:109E7000F6F7DDF90646F6F735FD044622460B46B1
:109E800018A0FDF7A7FF11480068F6F72BFD044660
:109E900022460B4618A0FDF79DFF01211C48F8F74C
:109EA00098FA002802D11BA0FDF794FF01211C485D
:109EB000F8F78FFA002802D11AA0FDF78BFF70BDCA
:109EC000B80300201027000001010020D403002067
:109ED000616C6B6120766363203D252E32660D0A2E
:109EE000000000006C69746820766363203D2025C3
:109EF0002E3266200D0A00006D63755F74656D700B
:109F00006572617475726520252E31660D0A000038
:109F100000FC0140616C6B61206C6F73650D0A0081
:109F2000C00C00406C697468206C6F73650D0A008A
:109F300010B5FCF742FAF9F78BFEF9F707FD10BDF3
:109F4000F0B585B00020294908607D24E400204652
:109F5000604301462648F6F7D1F8054629462046D3
:109F6000FDF7B6FA002705E00120FEF78FFFF9F7AD
:109F700069F87F1C7D20C0008742F5D30020F7F7E9
:109F80001DFA1A4806686E432046F6F7F2FB0746AC
:109F90003046F6F7EEFB39460190F6F7D1F903901B
:109FA00014490398F6F7C4F912490190F6F705FA37
:109FB00007461149F6F7C4F902900398F6F792FCA8
:109FC00002460B46019100900CA0FDF703FF02989A
:109FD000F6F788FC02460B46019100900FA0FDF7B2
:109FE000F9FE0120F7F7EAF905B0F0BDB003002053
:109FF000001BB700001B374B0000C8424D65617362
:10A0000075726564204672657175656E63793A2074
:10A01000252E326620487A0A000000004572726FD1
:10A02000722050657263656E746167653A20252EF3
:10A03000326625250A00000010B586B004460120CE
:10A04000F7F790FA0120FCF79FFE0020FCF78CFE4A
:10A050000120FCF777FE0020FDF79CFE0020F7F7BB
:10A0600081FA02200190029400206946087304904E
:10A070000320059001A8FCF767FDF8F7E3FF30BF68
:10A08000F8F7E0FF0020FCF75DFE06B010BD000011
:10A0900010B5012149020448F8F79BF9002801D1C5
:10A0A000012010BD0020FCE7000D004001464800E3
:10A0B0000A06D20F1B235A435040C0B27047637C3C
:10A0C000777BF26B6FC53001672BFED7AB76CA8208
:10A0D000C97DFA5947F0ADD4A2AF9CA472C0B7FDB8
:10A0E0009326363FF7CC34A5E5F171D8311504C776
:10A0F00023C31896059A071280E2EB27B2750983ED
:10A100002C1A1B6E5AA0523BD6B329E32F8453D18D
:10A1100000ED20FCB15B6ACBBE394A4C58CFD0EF82
:10A12000AAFB434D338545F9027F503C9FA851A3BC
:10A13000408F929D38F5BCB6DA2110FFF3D2CD0CDA
:10A1400013EC5F974417C4A77E3D645D197360816B
:10A150004FDC222A908846EEB814DE5E0BDBE0323C
:10A160003A0A4906245CC2D3AC629195E479E7C807
:10A17000376D8DD54EA96C56F4EA657AAE08BA787B
:10A18000252E1CA6B4C6E8DD741F4BBD8B8A703E1D
:10A19000B5664803F60E613557B986C11D9EE1F8D4
:10A1A000981169D98E949B1E87E9CE5528DF8CA122
:10A1B000890DBFE6426841992D0FB054BB16520974
:10A1C0006AD53036A538BF40A39E81F3D7FB7CE328
:10A1D00039829B2FFF87348E4344C4DEE9CB547B06
:10A1E0009432A6C2233DEE4C950B42FAC34E082E84
:10A1F000A16628D924B2765BA2496D8BD12572F86D
:10A20000F66486689816D4A45CCC5D65B6926C70D2
:10A210004850FDEDB9DA5E154657A78D9D8490D85C
:10A22000AB008CBCD30AF7E45805B8B34506D02C74
:10A230001E8FCA3F0F02C1AFBD0301138A6B3A9153
:10A2400011414F67DCEA97F2CFCEF0B4E67396ACDB
:10A250007422E7AD3585E2F937E81C75DF6E47F10A
:10A260001A711D29C5896FB7620EAA18BE1BFC564C
:10A270003E4BC6D279209ADBC0FE78CD5AF41FDD62
:10A28000A8338807C731B11210592780EC5F60519D
:10A290007FA919B54A0D2DE57A9F93C99CEFA0E0DF
:10A2A0003B4DAE2AF5B0C8EBBB3C83539961172BED
:10A2B000047EBA77D626E169146355210C7D8D01A1
:10A2C000020408102040801B366CD8AB4D9A2F5EDC
:10A2D000BC63C697356AD4B37DFAEFC5913972E491
:10A2E000D3BD61C29F254A943366CC831D3A74E87E
:10A2F000CB8D01020408102040801B366CD8AB4D7A
:10A300009A2F5EBC63C697356AD4B37DFAEFC591C8
:10A310003972E4D3BD61C29F254A943366CC831D54
:10A320003A74E8CB8D01020408102040801B366C83
:10A33000D8AB4D9A2F5EBC63C697356AD4B37DFA0D
:10A34000EFC5913972E4D3BD61C29F254A9433664B
:10A35000CC831D3A74E8CB8D0102040810204080A4
:10A360001B366CD8AB4D9A2F5EBC63C697356AD44A
:10A37000B37DFAEFC5913972E4D3BD61C29F254A1E
:10A38000943366CC831D3A74E8CB8D010204081027
:10A390002040801B366CD8AB4D9A2F5EBC63C697AD
:10A3A000356AD4B37DFAEFC5913972E4D3BD61C289
:10A3B0009F254A943366CC831D3A74E8CB00000095
:10A3C00060A6000050A50000D4A60000B8A60000BA
:10A3D000BCA40000E4A4000060AA00007CAA000065
:10A3E00080A50000ECA600001CA60000FCA5000053
:10A3F0000CA5000088A70000D0A7000000A700005F
:10A40000B8A8000080A80000E0A900008CA9000006
:10A4100038A9000060A900003CAA000018AA0000AA
:10A42000B0A9000008A8000038A6000060A700003E
:10A4300030A8000090A6000098AA000014A900000F
:10A44000ACA700003CA700005CA80000F0A800003A
:10A45000DCA50000C0A50000636D5F6261636B74E2
:10A46000726163655F61737365727400636D5F62CF
:10A4700061636B74726163655F6661756C74000023
:10A48000A0A40000A4A40000A8A40000ACA40000A4
:10A49000B8A40000B4A40000B0A400004CA50000C3
:10A4A000523020005231200052322000523320001E
:10A4B000504320004C522000523132003D3D3D3D82
:10A4C0003D3D3D3D3D3D3D20CFDFB3CCB6D1D5BB7D
:10A4D000D0C5CFA2203D3D3D3D3D3D3D3D3D3D3DB7
:10A4E000000000003D3D3D3D3D3D3D3D3D3D3D3D90
:10A4F00020D6F7B6D1D5BBD0C5CFA2203D3D3D3D3E
:10A500003D3D3D3D3D3D3D3D000000003D3D3D3D6F
:10A510003D3D3D3D3D3D3D3D3D3D3D3D3D3D3D3D6B
:10A520003D3D3D3D3D20BCC4B4E6C6F7D0C5CFA2FD
:10A53000203D3D3D3D3D3D3D3D3D3D3D3D3D3D3D68
:10A540003D3D3D3D3D3D3D3D3D3D000050535200B4
:10A55000B9CCBCFEC3FBB3C6A3BA2573A3ACD3B2BC
:10A56000BCFEB0E6B1BEBAC5A3BA2573A3ACC8EDB4
:10A57000BCFEB0E6B1BEBAC5A3BA257300000000A8
:10A58000B2E9BFB4B8FCB6E0BAAFCAFDB5F7D3C301
:10A59000D5BBD0C5CFA2A3ACC7EBD4CBD0D0A3BA88
:10A5A00061646472326C696E65202D6520257325A7
:10A5B00073202D61202D6620252E2A7300000000B7
:10A5C000B7A2C9FAD7DCCFDFB4EDCEF3B5C4B5D8A6
:10A5D000D6B7A3BA2530387800000000B7A2C9FA70
:10A5E000B4E6B4A2C6F7B9DCC0EDB4EDCEF3B5C4A1
:10A5F000B5D8D6B7A3BA253038780000D4DAD6D08B
:10A60000B6CFBBF2C2E3BBFABBB7BEB3CFC2B7A2F1
:10A61000C9FAB4EDCEF3D2ECB3A30000D4DACFDFA5
:10A62000B3CC28257329D6D0B7A2C9FAB4EDCEF39E
:10A63000D2ECB3A300000000B7A2C9FAD3C3B7A8F5
:10A64000B4EDCEF3A3ACD4ADD2F2A3BACAD4CDBC90
:10A65000C7D0BBBBB5BD2041524D20D7B4CCAC0058
:10A66000B4EDCEF3A3BACEDEB7A8BBF1C8A1D6F73E
:10A67000D5BBD0C5CFA2A3ACC7EBBCECB2E9D6F733
:10A68000D5BBB5C4CFE0B9D8C5E4D6C3000000003F
:10A69000B7A2C9FAD3C3B7A8B4EDCEF3A3ACD4AD77
:10A6A000D2F2A3BAC6F3CDBCD6B4D0D0B7C7B6D415
:10A6B000C6EBB7C3CECA0000D4DAD6D0B6CFBBF251
:10A6C000C2E3BBFABBB7BEB3CFC2B7A2C9FAB6CF1B
:10A6D000D1D40000D4DACFDFB3CC28257329D6D06B
:10A6E000B7A2C9FAB6CFD1D400000000BBF1C8A10F
:10A6F000BAAFCAFDB5F7D3C3D5BBCAA7B0DC00005B
:10A70000B7A2C9FAB4E6B4A2C6F7B9DCC0EDB4ED9D
:10A71000CEF3A3ACD4ADD2F2A3BAC6F3CDBCB4D3BE
:10A72000B2BBD4CAD0EDB7C3CECAB5C4C7F8D3F252
:10A73000B6C1A1A2D0B4CAFDBEDD0000B7A2C9FA5D
:10A74000B5F7CAD4B4EDCEF3A3ACD4ADD2F2A3BA6C
:10A75000CAFDBEDDBCE0B2E2B5E3C6A5C5E40000BB
:10A76000B7A2C9FAD3C3B7A8B4EDCEF3A3ACD4ADA6
:10A77000D2F2A3BACEDED0A7B5C4D2ECB3A3B7B59C
:10A78000BBD8C2EB00000000B7A2C9FAD3B2B4ED47
:10A79000CEF3A3ACD4ADD2F2A3BAC8A1D6D0B6CF73
:10A7A000CFF2C1BFCAB1B3F6B4ED0000B7A2C9FA87
:10A7B000B5F7CAD4B4EDCEF3A3ACD4ADD2F2A3BAFC
:10A7C000D6B4D0D020424B505420D6B8C1EE0000B1
:10A7D000B7A2C9FAB4E6B4A2C6F7B9DCC0EDB4EDCD
:10A7E000CEF3A3ACD4ADD2F2A3BAC6F3CDBCB4D3EE
:10A7F000B2BBD4CAD0EDB7C3CECAB5C4C7F8D3F282
:10A80000C8A1D6B8C1EE0000B7A2C9FAD3C3B7A891
:10A81000B4EDCEF3A3ACD4ADD2F2A3BAC6F3CDBCA3
:10A82000D6B4D0D0CEB4B6A8D2E5D6B8C1EE00002A
:10A83000B7A2C9FAD3C3B7A8B4EDCEF3A3ACD4ADD5
:10A84000D2F2A3BAC6F3CDBCD6B4D0D0D0ADB4A6A4
:10A85000C0EDC6F7D6B8C1EE00000000B7A2C9FA35
:10A86000B5F7CAD4B4EDCEF3A3ACD4ADD2F2A3BA4B
:10A87000B7A2C9FACFF2C1BFB2B6BBF10000000067
:10A88000B7A2C9FAB4E6B4A2C6F7B9DCC0EDB4ED1C
:10A89000CEF3A3ACD4ADD2F2A3BAC8EBD5BBCAB148
:10A8A000C6F3CDBCB7C3CECAB2BBB1BBD4CAD0ED20
:10A8B000B5C4C7F8D3F20000B7A2C9FAB4E6B4A28F
:10A8C000C6F7B9DCC0EDB4EDCEF3A3ACD4ADD2F293
:10A8D000A3BAB3F6D5BBCAB1C6F3CDBCB7C3CECA13
:10A8E000B2BBB1BBD4CAD0EDB5C4C7F8D3F2000037
:10A8F000B7A2C9FAB5F7CAD4B4EDCEF3A3ACD4ADC0
:10A90000D2F2A3BACDE2B2BFB5F7CAD4C7EBC7F350
:10A9100000000000B7A2C9FAB5F7CAD4B4EDCEF36F
:10A92000A3ACD4ADD2F2A3BA4E56494320CDA3BBBB
:10A93000FAC7EBC7F3000000B7A2C9FAD7DCCFDF34
:10A94000B4EDCEF3A3ACD4ADD2F2A3BABEABC8B7CC
:10A95000B5C4CAFDBEDDD7DCCFDFB4EDCEF3000059
:10A96000B7A2C9FAD7DCCFDFB4EDCEF3A3ACD4AD38
:10A97000D2F2A3BAB2BBBEABC8B7B5C4CAFDBEDD86
:10A98000D7DCCFDFB4EDCEF300000000B7A2C9FAE8
:10A99000D7DCCFDFB4EDCEF3A3ACD4ADD2F2A3BA03
:10A9A000D6B8C1EED7DCCFDFB4EDCEF300000000A7
:10A9B000B7A2C9FAD7DCCFDFB4EDCEF3A3ACD4ADE8
:10A9C000D2F2A3BAB6E8D0D4B1A3B4E6B8A1B5E345
:10A9D000D7B4CCACCAB1B7A2C9FAB4EDCEF300007B
:10A9E000B7A2C9FAB4E6B4A2C6F7B9DCC0EDB4EDBB
:10A9F000CEF3A3ACD4ADD2F2A3BAB6E8D0D4B1A30F
:10AA0000B4E6B8A1B5E3D7B4CCACCAB1B7A2C9FA21
:10AA1000B4EDCEF300000000B7A2C9FAD7DCCFDF57
:10AA2000B4EDCEF3A3ACD4ADD2F2A3BAC8EBD5BB90
:10AA3000CAB1B7A2C9FAB4EDCEF30000B7A2C9FA01
:10AA4000D7DCCFDFB4EDCEF3A3ACD4ADD2F2A3BA52
:10AA5000B3F6D5BBCAB1B7A2C9FAB4EDCEF30000C4
:10AA6000B4EDCEF3A3BACFDFB3CCD5BB28253038B5
:10AA70007829B7A2C9FAD2E7B3F60000B4EDCEF355
:10AA8000A3BAD6F7D5BB282530387829B7A2C9FA9A
:10AA9000D2E7B3F600000000B7A2C9FAD3C3B7A843
:10AAA000B4EDCEF3A3ACD4ADD2F2A3BAC6F3CDBC11
:10AAB000D6B4D0D0B3FD203020B2D9D7F7000000F3
:10AAC000E0AA00000000002048060000740B00000F
:10AAD00020AD000048060020C06D0000767E00001A
:10AAE000417205259632B8411AF00417784D55EC9D
:10AAF000DC2517276C5169AA26123C1401A0051306
:10AB000010010216101A0A31110009A108070605E2
:10AB1000040302017208BB0101AC826485D002D03B
:10AB2000020916CE16200102603F137F068E0832FE
:10AB3000011F060E1A3054521023448013030213CF
:10AB400028011320634A050912014A0809214A090C
:10AB50000912034A0B09227012023A2A1B4A010900
:10AB600012954A04092A963F290912974A06092A8A
:10AB70009036290912914A0C0912924A0D09129332
:10AB80004A0E0912944A0F09198F12021A2C092A27
:10AB9000115A290912124A02092A13A229092A1450
:10ABA0006C29092A156C29092A05AB290919911262
:10ABB000021A2E092A213F29092A223F29092A237C
:10ABC0003F29092A243F29092A303F29092A31AB84
:10ABD000290912324A07092A255129092A26FC295E
:10ABE0000912274A0A092A28CF29092A29CF29091F
:10ABF0002A41751A30092A427529092A43752909FB
:10AC00002A447529092A457529092A467529092AD8
:10AC1000477529092A407529092A487529092A49A9
:10AC20007529092A507529092A517529092A666C3E
:10AC30001A32092A066C29092A336C29092A606C00
:10AC400029092A616C29092A626C29092A656C295B
:10AC5000092A646C29092A716C290942011A3409EC
:10AC60001202190B29091A0362390912044A03094D
:10AC700012054A040912064A080912074A0909126C
:10AC8000084A0A0912094A0B09120A4A0C09012C3E
:10AC9000169901030DADA40E57431958521E2AB43C
:10ACA00099B904214B4816605A98085AC0085AE8C6
:10ACB00008016E0334803FA40A3412480F554647FA
:10ACC0003232304731304C4E565A20010114142094
:10ACD0002301021D104009666666416666864108CA
:10ACE00009109A999941CDCCCC3DAB2302431A0867
:10ACF000044B8C42042910690CC92C1228123216FC
:10AD0000F6FFF1FF2854F1FF321A320A811A640E5D
:10AD100041199449696961012603670101D3127AD7
:04000005000000C136
:00000001FF
